:020000040000FA
:0408000090EF0BF07A
:1008100003B273EF05F0F2B491EF05F09EB099EFDB
:1008200005F09EB2A1EF05F0F2A81AEF04F0F2B2C3
:1008300021EF04F0F2B01FEF04F03FEF0BF0F2965F
:10084000F290CD90F2929EA02BEF04F00101533F65
:100850002BEF04F0542BB2C1B6F1B3C1B7F1B4C160
:10086000B8F1B5C1B9F1AEC1B2F1AFC1B3F1B0C128
:10087000B4F1B1C1B5F1AAC1AEF1ABC1AFF1ACC138
:10088000B0F1ADC1B1F1A6C1AAF1A7C1ABF1A8C148
:10089000ACF1A9C1ADF1A2C1A6F1A3C1A7F1A4C158
:1008A000A8F1A5C1A9F19EC1A2F19FC1A3F1A0C168
:1008B000A4F1A1C1A5F19AC19EF19BC19FF19CC178
:1008C000A0F19DC1A1F1CECF9AF1CFCF9BF153C141
:1008D0009CF154C19DF1CF6ACE6A0101536B546BF8
:1008E0009E90CD800FBC0F8E0FBA7AEF04F00F8A66
:1008F0003FEF0BF013880F8C0FBEB7EF04F09AC1D7
:100900009EF19BC19FF19CC1A0F19DC1A1F19EC12F
:10091000A2F19FC1A3F1A0C1A4F1A1C1A5F1A2C1FF
:10092000A6F1A3C1A7F1A4C1A8F1A5C1A9F1A6C1CF
:10093000AAF1A7C1ABF1A8C1ACF1A9C1ADF1AAC19F
:10094000AEF1ABC1AFF1ACC1B0F1ADC1B1F1AEC16F
:10095000B2F1AFC1B3F1B0C1B4F1B1C1B5F1B2C13F
:10096000B6F1B3C1B7F1B4C1B8F1B5C1B9F1010184
:100970005E6B5F6B606B616B9A515E279B515F236F
:100980009C5160239D5161239E515E279F515F239F
:10099000A0516023A1516123A2515E27A3515F237F
:1009A000A4516023A5516123A6515E27A7515F235F
:1009B000A8516023A9516123AA515E27AB515F233F
:1009C000AC516023AD516123AE515E27AF515F231F
:1009D000B0516023B1516123B2515E27B3515F23FF
:1009E000B4516023B5516123B6515E27B7515F23DF
:1009F000B8516023B9516123D8900101613360334C
:100A00005F335E33D8900101613360335F335E330F
:100A1000D8900101613360335F335E3300C10CF164
:100A200001C10DF102C10EF103C10FF104C110F1BA
:100A300005C111F106C112F107C113F108C114F18A
:100A400009C115F10AC116F10BC117F134C135F115
:100A500011B836EF05F00101620E046F010E056F4B
:100A6000000E066F000E076F3FEF05F00101A70EA5
:100A7000046F020E056F000E066F000E076F5EC159
:100A800000F15FC101F160C102F161C103F164ECE9
:100A90002FF003BF04D01CBE02D01CA0108C11A0EC
:100AA00057EF05F010BA57EF05F00F80108A0CC110
:100AB00000F10DC101F10EC102F10FC103F110C12E
:100AC00004F111C105F112C106F113C107F114C1FE
:100AD00008F115C109F116C10AF117C10BF135C1B1
:100AE00034F13FEF0BF00392ABB2AB98AB8803014C
:100AF00003EE00F080517F0BE92604C0EFFF802B4E
:100B00008151805D700BD8A48B8200008051815D83
:100B1000700BD8A48B9281518019D8B407903FEF05
:100B20000BF0F2940101453F3FEF0BF0462B3FEFF6
:100B30000BF09E900101533F3FEF0BF0542B3FEF22
:100B40000BF09E9211B841EF08F0040066A1A9EFE6
:100B500005F08BB4B3EF05F010ACB3EF05F08B8468
:100B6000109CB4EF05F08B94077C07ACCFEF05F039
:100B7000C274C2B4C9EF05F0C3CFB7F5C4CFB8F59E
:100B80000501D890B833B733D890B833B733D0EF26
:100B900005F0C3CF55F1C4CF56F1D0EF05F0C282B6
:100BA00007B442EF06F047C14BF148C14CF149C1CF
:100BB0004DF14AC14EF15EC162F15FC163F160C1A6
:100BC00064F161C165F113A8E8EF05F0138C139887
:100BD0009AC1BAF19BC1BBF19CC1BCF19DC1BDF1F1
:100BE0009EC1BEF19FC1BFF1A0C1C0F1A1C1C1F1C1
:100BF000A2C1C2F1A3C1C3F1A4C1C4F1A5C1C5F191
:100C0000A6C1C6F1A7C1C7F1A8C1C8F1A9C1C9F160
:100C1000AAC1CAF1ABC1CBF1ACC1CCF1ADC1CDF130
:100C2000AEC1CEF1AFC1CFF1B0C1D0F1B1C1D1F100
:100C3000B2C1D2F1B3C1D3F1B4C1D4F1B5C1D5F1D0
:100C4000B6C1D6F1B7C1D7F1B8C1D8F1B9C1D9F1A0
:100C5000B7C5B9F5B8C5BAF5B9C5BBF5BAC5BCF5E0
:100C6000010155515B2756515C23E86A5D230E2E26
:100C700042EF06F05CC157F15DC158F15B6B5C6BF4
:100C80005D6B078E0201002F3FEF0BF03C0E006FF3
:100C90001D50E00BE00AE86612881BBE02D01BB4B0
:100CA000108E00C10CF101C10DF102C10EF103C1A2
:100CB0000FF104C110F105C111F106C112F107C114
:100CC00013F108C114F109C115F10AC116F10BC1E4
:100CD00017F134C135F181AAAAEF06F037A0F5EF7C
:100CE00006F005012F51000AD8B438EF07F00501CE
:100CF0002F51010AD8B4B4EF06F005012F51020AB2
:100D0000D8B4F5EF06F005012F51030AD8B4F5EF7A
:100D100006F005012F51040AD8B4F5EF06F00501DD
:100D20002F51050AD8B4F5EF06F005012F51060A38
:100D3000D8B4F5EF06F005012F51070AD8B4F5EF46
:100D400006F005012F51320AD8B4B2EF06F02F6B2E
:100D500038EF07F000011650030AD8B4F5EF06F09B
:100D600038EF07F038EF07F005015767BFEF06F0DF
:100D70005867BFEF06F05967BFEF06F05A67C3EF39
:100D800006F038EF07F05BC500F15CC501F15DC509
:100D900002F15EC503F10101010E046F000E056F43
:100DA000000E066F000E076F64EC2FF000C15BF5BC
:100DB00001C15CF502C15DF503C15EF5010100678B
:100DC000E9EF06F00167E9EF06F00267E9EF06F0E8
:100DD000036738EF07F057C55BF558C55CF559C593
:100DE0005DF55AC55EF522EF07F00FBE0AEF07F07A
:100DF00010A00FEF07F00101476706EF07F0486703
:100E000006EF07F0496706EF07F04A670AEF07F0B9
:100E10000FEF07F007AE0FEF07F022EF07F0050125
:100E2000312F38EF07F03C0E316F302F38EF07F0DD
:100E30000101000E626FE00E636FA50E646F010E7C
:100E4000656F138800011650000AD8B430EF07F020
:100E500000011650030AD8B435EF07F038EF07F059
:100E60000001010E166E38EF07F00001040E166E39
:100E70000501666B37B73EEF07F066810CC100F1E4
:100E80000DC101F10EC102F10FC103F110C104F156
:100E900011C105F112C106F113C107F114C108F126
:100EA00015C109F116C10AF117C10BF135C134F1B1
:100EB00000C10CF101C10DF102C10EF103C10FF12E
:100EC00004C110F105C111F106C112F107C113F1FE
:100ED00008C114F109C115F10AC116F10BC117F1CE
:100EE00034C135F101018E677DEF07F08F677DEF2B
:100EF00007F090677DEF07F0916781EF07F0B2EFA1
:100F000007F092C100F193C101F194C102F195C1C2
:100F100003F10101010E046F000E056F000E066F54
:100F2000000E076F64EC2FF000C192F101C193F144
:100F300002C194F103C195F101010067A7EF07F029
:100F40000167A7EF07F00267A7EF07F00367B2EFAB
:100F500007F08EC192F18FC193F190C194F191C1CC
:100F600095F10F80D57ED5BE6ED0D6CF47F1D7CFC5
:100F700048F145C149F1E86AE8CF4AF1138A1CBE3D
:100F800002D01CA0108C109047C100F148C101F1A3
:100F900049C102F14AC103F101010A0E046F000EBA
:100FA000056F000E066F000E076F64EC2FF003AFA5
:100FB0001080010154A7E9EF07F00F9A0F9C0F9ED4
:100FC0000101000E5E6F600E5F6F3D0E606F080ED8
:100FD000616F010147BFF9EF07F04867F9EF07F0CC
:100FE0004967F9EF07F04A67F9EF07F0F2881EEF5B
:100FF00008F0F2985E6B5F6B606B616B9A6B9B6B3A
:101000009C6B9D6B9E6B9F6BA06BA16BA26BA36B8C
:10101000A46BA56BA66BA76BA86BA96BAA6BAB6B3C
:10102000AC6BAD6BAE6BAF6BB06BB16BB26BB36BEC
:10103000B46BB56BB66BB76BB86BB96BD76AD66A66
:101040000101456B466B0CC100F10DC101F10EC1F0
:1010500002F10FC103F110C104F111C105F112C178
:1010600006F113C107F114C108F115C109F116C148
:101070000AF117C10BF135C134F13FEF0BF03FEF2F
:101080000BF00201002FA3EF0AF0D59ED6CF47F157
:10109000D7CF48F145C149F1E86AE8CF4AF1138A50
:1010A000D76AD66A0101456B466BD58E1D50E00BA1
:1010B000E00AE86612881BBE02D01BB4108E1AAE7E
:1010C0001F8C00C10CF101C10DF102C10EF103C171
:1010D0000FF104C110F105C111F106C112F107C1F0
:1010E00013F108C114F109C115F10AC116F10BC1C0
:1010F00017F134C135F10FA0109A11B88BEF08F039
:101100000101620E046F010E056F000E066F000EE6
:10111000076F94EF08F00101A70E046F020E056F30
:10112000000E066F000E076F47C100F148C101F1C4
:1011300049C102F14AC103F164EC2FF003BFA7EFEC
:1011400008F01CBE02D01CA0108C11B00F800CC186
:1011500000F10DC101F10EC102F10FC103F110C187
:1011600004F111C105F112C106F113C107F114C157
:1011700008F115C109F116C10AF117C10BF135C10A
:1011800034F102013C0E006F00C10CF101C10DF100
:1011900002C10EF103C10FF104C110F105C111F13B
:1011A00006C112F107C113F108C114F109C115F10B
:1011B0000AC116F10BC117F134C135F181AA1DEF37
:1011C00009F037A068EF09F005012F51000AD8B4E3
:1011D000ABEF09F005012F51010AD8B427EF09F050
:1011E00005012F51020AD8B468EF09F005012F510B
:1011F000030AD8B468EF09F005012F51040AD8B4E6
:1012000068EF09F005012F51050AD8B468EF09F01D
:1012100005012F51060AD8B468EF09F005012F51D6
:10122000070AD8B468EF09F005012F51320AD8B483
:1012300025EF09F02F6BABEF09F000011650030A00
:10124000D8B468EF09F0ABEF09F0ABEF09F0050196
:10125000576732EF09F0586732EF09F0596732EFFC
:1012600009F05A6736EF09F0ABEF09F05BC500F102
:101270005CC501F15DC502F15EC503F10101010E1E
:10128000046F000E056F000E066F000E076F64EC12
:101290002FF000C15BF501C15CF502C15DF503C132
:1012A0005EF5010100675CEF09F001675CEF09F092
:1012B00002675CEF09F00367ABEF09F057C55BF518
:1012C00058C55CF559C55DF55AC55EF595EF09F051
:1012D0000FBE7DEF09F010A082EF09F00101476712
:1012E00079EF09F0486779EF09F0496779EF09F07C
:1012F0004A677DEF09F082EF09F007AE82EF09F04F
:1013000095EF09F00501312FABEF09F03C0E316F7D
:10131000302FABEF09F00101000E626FE00E636F3A
:10132000A50E646F010E656F138800011650000A48
:10133000D8B4A3EF09F000011650030AD8B4A8EFFF
:1013400009F0ABEF09F00001010E166EABEF09F0EA
:101350000001040E166E0501666B37B7B1EF09F098
:1013600066810CC100F10DC101F10EC102F10FC186
:1013700003F110C104F111C105F112C106F113C14D
:1013800007F114C108F115C109F116C10AF117C11D
:101390000BF135C134F100C10CF101C10DF102C1F5
:1013A0000EF103C10FF104C110F105C111F106C125
:1013B00012F107C113F108C114F109C115F10AC1F5
:1013C00016F10BC117F134C135F101018E67F0EF51
:1013D00009F08F67F0EF09F09067F0EF09F091677F
:1013E000F4EF09F025EF0AF092C100F193C101F189
:1013F00094C102F195C103F10101010E046F000EC9
:10140000056F000E066F000E076F64EC2FF000C131
:1014100092F101C193F102C194F103C195F101016F
:1014200000671AEF0AF001671AEF0AF002671AEF75
:101430000AF0036725EF0AF08EC192F18FC193F194
:1014400090C194F191C195F10F80109047C100F1C6
:1014500048C101F149C102F14AC103F101010A0E7B
:10146000046F000E056F000E066F000E076F64EC30
:101470002FF003AF1080010154A74BEF0AF00F9A31
:101480000F9C0F9E0101000E5E6F600E5F6F3D0EA0
:10149000606F080E616F47C100F148C101F149C199
:1014A00002F14AC103F10101140E046F050E056F2C
:1014B000000E066F000E076F64EC2FF003AF64EFB1
:1014C0000AF0F28889EF0AF0F2985E6B5F6B606B4E
:1014D000616B9A6B9B6B9C6B9D6B9E6B9F6BA06B08
:1014E000A16BA26BA36BA46BA56BA66BA76BA86B80
:1014F000A96BAA6BAB6BAC6BAD6BAE6BAF6BB06B30
:10150000B16BB26BB36BB46BB56BB66BB76BB86BDF
:10151000B96B0CC100F10DC101F10EC102F10FC197
:1015200003F110C104F111C105F112C106F113C19B
:1015300007F114C108F115C109F116C10AF117C16B
:101540000BF135C134F104008BB4AEEF0AF010ACEE
:10155000AEEF0AF08B84109CAFEF0AF08B94077CFF
:1015600007ACCAEF0AF0C274C2B4C4EF0AF0C3CF2A
:10157000B7F5C4CFB8F50501D890B833B733D890D4
:10158000B833B733CBEF0AF0C3CF55F1C4CF56F120
:10159000CBEF0AF0C28207B43DEF0BF047C14BF12D
:1015A00048C14CF149C14DF14AC14EF15EC162F1F1
:1015B0005FC163F160C164F161C165F113A8E3EF3C
:1015C0000AF0138C13989AC1BAF19BC1BBF19CC16C
:1015D000BCF19DC1BDF19EC1BEF19FC1BFF1A0C1D3
:1015E000C0F1A1C1C1F1A2C1C2F1A3C1C3F1A4C1A3
:1015F000C4F1A5C1C5F1A6C1C6F1A7C1C7F1A8C173
:10160000C8F1A9C1C9F1AAC1CAF1ABC1CBF1ACC142
:10161000CCF1ADC1CDF1AEC1CEF1AFC1CFF1B0C112
:10162000D0F1B1C1D1F1B2C1D2F1B3C1D3F1B4C1E2
:10163000D4F1B5C1D5F1B6C1D6F1B7C1D7F1B8C1B2
:10164000D8F1B9C1D9F1B7C5B9F5B8C5BAF5B9C5B9
:10165000BBF5BAC5BCF5010155515B2756515C235A
:10166000E86A5D230E2E3DEF0BF05CC157F15DC1C2
:1016700058F15B6B5C6B5D6B078E3FEF0BF002C04C
:10168000E0FF005001C0D8FF1000A6B245EF0BF0FC
:101690000CC0A9FF0BC0A8FFA69EA69CA684F29E24
:1016A000550EA76EAA0EA76EA682F28EA694A6B2BB
:1016B00057EF0BF00C2A1200A96EA69EA69CA680DE
:1016C000A8500C2A120004012C0E826FD3EC0EF0ED
:1016D0005FEC30F00C505CEC0BF0E8CF00F10C50FC
:1016E0005CEC0BF0E8CF01F101AF7CEF0BF00101F6
:1016F000FF0E026FFF0E036F02EC30F0296788EFD8
:101700000BF00401200E826FD3EC0EF08DEF0BF086
:1017100004012D0E826FD3EC0EF00CEC2EF01200B3
:10172000376A076A0F6A106A116A126A136A156AC1
:10173000166A0F010D0EC16E860EC06E030EC26ECC
:101740000F01680E896E130E926E080E8A6EF30EEC
:10175000936E8B6A900E946EC80E5CEC0BF0E8CF23
:10176000E8FF1098E8A0108810A805D00E0E256E8E
:101770008E0E266E04D00F0E256E8F0E266EF7ECA1
:1017800030F0F18EF19EFC0E5CEC0BF0E8CF0BF02C
:101790000BA011800BA211820BA411840BA811883D
:1017A000C90E5CEC0BF0E8CF1AF0CA0E5CEC0BF043
:1017B000E8CF1BF0CB0E5CEC0BF0E8CF1CF0CC0EAE
:1017C0005CEC0BF0E8CF1DF0FB0E5CEC0BF0E8CF0F
:1017D00038F0CE0E5CEC0BF0E8CF14F0CD0E5CECE4
:1017E0000BF0E8CF36F01F6A206A0E6A01015B6BCE
:1017F0005C6B5D6B576B586BF29A0101476B486BE2
:10180000496B4A6B4B6B4C6B4D6B4E6B4F6B506B1C
:10181000516B526B456B466BD76AD66A0F01280E27
:10182000D56EF28A9D90B00ECD6E01015E6B5F6B3E
:10183000606B616B626B636B646B656B666B676B34
:10184000686B696B536B546BCF6ACE6A0F9A0F9CAF
:101850000F9E9D80760ECA6E9D8202013C0E006F27
:10186000CC6A160E5CEC0BF0E8CF00F1170E5CECC6
:101870000BF0E8CF01F1180E5CEC0BF0E8CF02F1B1
:10188000190E5CEC0BF0E8CF03F1010103AF63EF3D
:101890000CF05FEC30F0160E0C6E00C10BF045EC56
:1018A0000BF0170E0C6E01C10BF045EC0BF0180E8F
:1018B0000C6E02C10BF045EC0BF0190E0C6E03C15F
:1018C0000BF045EC0BF000C18EF101C18FF102C1AC
:1018D00090F103C191F100C192F101C193F102C1F4
:1018E00094F103C195F11A0E5CEC0BF0E8CF00F116
:1018F0001B0E5CEC0BF0E8CF01F11C0E5CEC0BF066
:10190000E8CF02F11D0E5CEC0BF0E8CF03F1010112
:1019100003AFB9EF0CF05FEC30F01A0E0C6E00C1A3
:101920000BF045EC0BF01B0E0C6E01C10BF045ECFF
:101930000BF01C0E0C6E02C10BF045EC0BF01D0EF3
:101940000C6E03C10BF045EC0BF01A0E5CEC0BF0C7
:10195000E8CF00F11B0E5CEC0BF0E8CF01F11C0EA0
:101960005CEC0BF0E8CF02F11D0E5CEC0BF0E8CF65
:1019700003F100C196F101C197F102C198F103C1D1
:1019800099F1240EAC6E900EAB6E240EAC6E080E68
:10199000B86E000EB06E1F0EAF6E0401806B816BCF
:1019A0000F01900EAB6E0F019D8A0301806B816B5E
:1019B000C26B8B929CEC35F09CEC35F072EC37F0FE
:1019C0007AEC33F0200E5CEC0BF0E8CF2FF505013C
:1019D0002F51FF0AD8A4F4EF0CF02F6B200E0C6EE1
:1019E0002FC50BF045EC0BF00501010E306F3C0EDE
:1019F000316F250E5CEC0BF0E8CF00F1260E5CECAD
:101A00000BF0E8CF01F1270E5CEC0BF0E8CF02F110
:101A1000280E5CEC0BF0E8CF03F1010103AF2BEFD4
:101A20000DF05FEC30F0250E0C6E00C10BF045ECB4
:101A30000BF0260E0C6E01C10BF045EC0BF0270EDF
:101A40000C6E02C10BF045EC0BF0280E0C6E03C1BE
:101A50000BF045EC0BF000C157F501C158F502C180
:101A600059F503C15AF500C15BF501C15CF502C12E
:101A70005DF503C15EF5290E5CEC0BF0E8CF5FF578
:101A8000050160515F5DD8A05FC560F5210E5CEC7B
:101A90000BF0E8CF00F1220E5CEC0BF0E8CF01F187
:101AA000230E5CEC0BF0E8CF02F1240E5CEC0BF0A3
:101AB000E8CF03F1010103AF8CEF0DF05FEC30F0E4
:101AC000210E0C6E00C10BF045EC0BF0220E0C6EDB
:101AD00001C10BF045EC0BF0230E0C6E02C10BF0B4
:101AE00045EC0BF0240E0C6E03C10BF045EC0BF033
:101AF000210E5CEC0BF0E8CF00F1220E5CEC0BF059
:101B0000E8CF01F1230E5CEC0BF0E8CF02F1240EDC
:101B10005CEC0BF0E8CF03F100C161F501C162F5A7
:101B200002C163F503C164F5C2EC32F0A8EC31F0F8
:101B300000EC31F037A0FDEF0DF005012F51020A46
:101B400016E005012F51030A19E005012F51040A7F
:101B500024E005012F51050A2BE005012F51060A4B
:101B600039E005012F51070A3FE0FDEF0DF0602F2E
:101B7000FAEF0DF05FC560F5FDEF0DF0B0C500F1B7
:101B800001010F0E001701010051000A36E00101AA
:101B90000051050A32E0FAEF0DF0B0C500F1010185
:101BA0000F0E001701010051000A27E0FAEF0DF0B7
:101BB0000501B051000A21E00501B051150A1DE0F0
:101BC0000501B051300A19E00501B051450A15E090
:101BD000FAEF0DF00501B051000A0FE00501B05118
:101BE000300A0BE0FAEF0DF00501B051000A05E0F4
:101BF000FAEF0DF081BAB1EF37F007900001F28EE5
:101C0000F28C12AE03D012BC52EF19F007B0A2EF63
:101C10002CF00FB09EEF25F010BE9EEF25F012B80D
:101C20009EEF25F000011650010AD8B4B9EF1DF05F
:101C300081BA23EF0EF000011650040AD8B4FEEF6B
:101C40001BF029EF0EF000011650040AD8B4E4EF9F
:101C50001DF00301805181197F0BD8B4A2EF2CF045
:101C600013EE00F081517F0BE126812BE7CFE8FFD7
:101C7000E00BD8B4A2EF2CF023EE82F0C2513F0B60
:101C8000D926E7CFDFFFC22BDF50780AD8A4A2EF16
:101C90002CF0078092C100F193C101F194C102F1CF
:101CA00095C103F10101040E046F000E056F000ED3
:101CB000066F000E076F64EC2FF000AF69EF0EF0B7
:101CC0000101030E926F000E936F000E946F000ED1
:101CD000956F03018251720AD8B41FEF25F082512B
:101CE000520AD8B41FEF25F08251750AD8B41FEFFD
:101CF00025F08251680AD8B4E7EF0EF08251630AEA
:101D0000D8B45CEF29F08251690AD8B4DDEF20F035
:101D100082517A0AD8B4F0EF21F08251490AD8B43E
:101D20007CEF20F08251500AD8B49AEF1FF0825114
:101D3000700AD8B4DDEF1FF08251540AD8B408EF0E
:101D400020F08251740AD8B44EEF20F08251410A3B
:101D5000D8B4ECEF0FF082514B0AD8B4E9EF0EF093
:101D600082516D0AD8B45CEF14F082514D0AD8B498
:101D700075EF14F08251730AD8B44FEF24F08251FA
:101D8000530AD8B4B4EF24F082514C0AD8B404EF0B
:101D900015F08251590AD8B4ADEF13F012AE01D04C
:101DA000128C93EF29F0040114EE00F080517F0BA8
:101DB000E12682C4E7FF802B120004010D0E826F22
:101DC000D3EC0EF00A0E826FD3EC0EF0120091EFFE
:101DD00029F004014B0E826FD3EC0EF004012C0E9F
:101DE000826FD3EC0EF081B802D036B630D003014A
:101DF0008351430AD8B42EEF0FF003018351630AD5
:101E0000D8B430EF0FF003018351520AD8B432EF47
:101E10000FF003018351720AD8B434EF0FF00301BD
:101E20008351470AD8B436EF0FF003018351670A94
:101E3000D8B438EF0FF003018351540AD8B43AEF05
:101E40000FF003018351740AD8B4AAEF0FF0030115
:101E50008351550AD8B43CEF0FF083D036807BD045
:101E6000369079D0368277D0369275D0368473D05A
:101E7000369471D036866FD084C330F185C331F18A
:101E800086C332F187C333F10101296BADEC30F029
:101E900024EC30F000C104F101C105F102C106F1EA
:101EA00003C107F1A0EC30F0200EF86EF76AF66A75
:101EB0000900F5CF2CF10900F5CF2DF10900F5CF80
:101EC0002EF10900F5CF2FF10900F5CF30F109000F
:101ED000F5CF31F10900F5CF32F10900F5CF33F13B
:101EE0000101296BADEC30F024EC30F064EC2FF004
:101EF0000101006783EF0FF0016783EF0FF00267C6
:101F000083EF0FF0036701D025D004014E0E826FDE
:101F1000D3EC0EF004016F0E826FD3EC0EF00401CF
:101F20004D0E826FD3EC0EF00401610E826FD3EC84
:101F30000EF00401740E826FD3EC0EF00401630EF8
:101F4000826FD3EC0EF00401680E826FD3EC0EF0BA
:101F500091EF29F03696CD0E0C6E36C00BF045ECA5
:101F60000BF0CD0E5CEC0BF0E8CF36F036B006D0BF
:101F70000401630E826FD3EC0EF005D00401430E12
:101F8000826FD3EC0EF036B206D00401720E826F6F
:101F9000D3EC0EF005D00401520E826FD3EC0EF09C
:101FA00036B406D00401670E826FD3EC0EF005D074
:101FB0000401470E826FD3EC0EF036B606D0040152
:101FC000740E826FD3EC0EF005D00401540E826FB4
:101FD000D3EC0EF091EF29F00401410E826FD3ECA7
:101FE0000EF003018351310AD8B4CDEF12F0030192
:101FF0008351320AD8B4FDEF11F003018351330A43
:10200000D8B486EF11F003018351340AD8B476EFC7
:1020100010F003018351350AD8B416EF10F0040113
:102020003F0E826FD3EC0EF091EF29F00301845143
:10203000300AD8B43CEF10F003018451310AD8B40F
:102040003FEF10F003018451650AD8B430EF10F06F
:1020500003018451640AD8B433EF10F040EF10F05C
:10206000389034EF10F03880FB0E0C6E38C00BF057
:1020700045EC0BF040EF10F08B9040EF10F08B80B0
:102080000401350E826FD3EC0EF004012C0E826F2A
:10209000D3EC0EF08BB054EF10F00401300E826FD1
:1020A000D3EC0EF059EF10F00401310E826FD3EC37
:1020B0000EF004012C0E826FD3EC0EF0FB0E5CECE4
:1020C0000BF0E8CF38F038A06DEF10F00401640E8B
:1020D000826FD3EC0EF072EF10F00401650E826F88
:1020E000D3EC0EF074EF10F091EF29F0CC0E5CEC15
:1020F0000BF0E8CF0BF004012C0E826FD3EC0EF046
:1021000003018451310AD8B49AEF10F003018451CD
:10211000300AD8B49CEF10F0030184514D0AD8B4B2
:10212000A6EF10F003018451540AD8B4ADEF10F0BB
:10213000C4EF10F08A8401D08A940BAE04D00BACAB
:1021400002D00BBA21D0E00E0B1218D01F0E0B16C6
:102150008539E844E00B0B1211D0E00E0B16A0EC11
:1021600030F085C332F186C333F10101296BADEC48
:1021700030F024EC30F000511F0B0B12CC0E0C6E23
:102180000BC00BF045EC0BF00401340E826FD3EC66
:102190000EF004012C0E826FD3EC0EF0CC0E5CEC32
:1021A0000BF0E8CF1DF08AB406D00401300E826F28
:1021B000D3EC0EF005D00401310E826FD3EC0EF09B
:1021C00004012C0E826FD3EC0EF01D38E840070B93
:1021D000E8CF82F40401300E8227D3EC0EF0040124
:1021E0002C0E826FD3EC0EF05FEC30F01D501F0B05
:1021F000E8CF00F102EC30F032C182F40401300E7D
:102200008227D3EC0EF033C182F40401300E822712
:10221000D3EC0EF004012C0E826FD3EC0EF05FECC9
:1022200030F030C000F100AF0BD0FF0E016FFF0E99
:10223000026FFF0E036F04012D0E826FD3EC0EF0C0
:1022400002EC30F031C182F40401300E8227D3EC6D
:102250000EF032C182F40401300E8227D3EC0EF06E
:1022600033C182F40401300E8227D3EC0EF0040156
:102270002C0E826FD3EC0EF05FEC30F02FC000F12B
:1022800002EC30F031C182F40401300E8227D3EC2D
:102290000EF032C182F40401300E8227D3EC0EF02E
:1022A00033C182F40401300E8227D3EC0EF0040116
:1022B0002C0E826FD3EC0EF05FEC30F031C000F1E9
:1022C00000AF0BD0FF0E016FFF0E026FFF0E036F0A
:1022D00004012D0E826FD3EC0EF002EC30F031C110
:1022E00082F40401300E8227D3EC0EF032C182F466
:1022F0000401300E8227D3EC0EF033C182F40401C6
:10230000300E8227D3EC0EF091EF29F0CB0E5CEC6F
:102310000BF0E8CF0BF004012C0E826FD3EC0EF023
:1023200003018451450AD8B4AAEF11F00301845186
:10233000440AD8B4ADEF11F003018451300AD8B487
:10234000B0EF11F003018451310AD8B4B4EF11F0A9
:10235000BFEF11F00B9EB9EF11F00B8EB9EF11F03A
:10236000FC0E0B16B9EF11F0FC0E0B160B80B9EF3B
:1023700011F0CB0E0C6E0BC00BF045EC0BF0040112
:10238000330E826FD3EC0EF004012C0E826FD3EC6F
:102390000EF0CB0E5CEC0BF0E8CF1CF01CBED8EFBF
:1023A00011F00401450E826FD3EC0EF0DDEF11F059
:1023B0000401440E826FD3EC0EF004012C0E826FE8
:1023C000D3EC0EF00401300E826FD3EC0EF004015A
:1023D0002C0E826FD3EC0EF01CB0F6EF11F004015E
:1023E000300E826FD3EC0EF0FBEF11F00401310ED2
:1023F000826FD3EC0EF091EF29F0CA0E5CEC0BF07B
:10240000E8CF0BF004012C0E826FD3EC0EF0030129
:102410008451450AD8B439EF12F003018451440ABB
:10242000D8B43CEF12F0030184514D0AD8B445EF03
:1024300012F003018451410AD8B43FEF12F00301B6
:102440008451460AD8B442EF12F003018451560A6F
:10245000D8B44DEF12F003018451500AD8B458EFAC
:1024600012F003018451520AD8B45BEF12F064EF0A
:1024700012F00B9E5EEF12F00B8E5EEF12F00B9CD3
:102480005EEF12F00B8C5EEF12F0FC0E0B1685C3A4
:10249000E8FF030B0B125EEF12F0C70E0B1685C39D
:1024A000E8FF070BE846E846E8460B125EEF12F03D
:1024B0000B845EEF12F00B945EEF12F0CA0E0C6EFE
:1024C0000BC00BF045EC0BF0CA0E5CEC0BF0E8CF48
:1024D0001BF00401320E826FD3EC0EF004012C0EBF
:1024E000826FD3EC0EF01BBE7DEF12F00401450E9F
:1024F000826FD3EC0EF082EF12F00401440E826F73
:10250000D3EC0EF004012C0E826FD3EC0EF01BC046
:10251000E8FF030BE8CF82F40401300E8227D3ECEE
:102520000EF004012C0E826FD3EC0EF01BBCA0EF5A
:1025300012F00401410E826FD3EC0EF0A5EF12F001
:102540000401460E826FD3EC0EF004012C0E826F54
:10255000D3EC0EF01BC0E8FF380BE842E842E8423B
:10256000E8CF82F40401300E8227D3EC0EF0040190
:102570002C0E826FD3EC0EF01BB4C6EF12F00401E8
:10258000520E826FD3EC0EF0CBEF12F00401500E1E
:10259000826FD3EC0EF091EF29F0C90E5CEC0BF0DA
:1025A000E8CF0BF004012C0E826FD3EC0EF0030188
:1025B0008451450AD8B4EBEF12F003018451440A68
:1025C000D8B4EEEF12F0030184514D0AD8B4F1EF04
:1025D00012F0FFEF12F00B9EF9EF12F00B8EF9EFF5
:1025E00012F0F80E0B1685C3E8FF070B0B12F9EF7C
:1025F00012F0C90E0C6E0BC00BF045EC0BF0040191
:10260000310E826FD3EC0EF004012C0E826FD3ECEE
:102610000EF0C90E5CEC0BF0E8CF1AF01ABE06D033
:102620000401450E826FD3EC0EF005D00401440E78
:10263000826FD3EC0EF004012C0E826FD3EC0EF0FF
:102640001AC0E8FF070BE8CF82F40401300E82279E
:10265000D3EC0EF004012C0E826FD3EC0EF0078049
:102660005FEC30F02BC0E8FF003B00430043030B5E
:1026700002EC30F033C182F40401300E8227D3EC37
:102680000EF004012C0E826FD3EC0EF05FEC30F0F4
:102690002BC001F1019F019D2CC000F1010102EC52
:1026A00030F02FC182F40401300E8227D3EC0EF0FB
:1026B00030C182F40401300E8227D3EC0EF031C118
:1026C00082F40401300E8227D3EC0EF032C182F482
:1026D0000401300E8227D3EC0EF033C182F40401E2
:1026E000300E8227D3EC0EF004012C0E826FD3EC57
:1026F0000EF05FEC30F02DC001F12EC000F1D8904B
:1027000001330033D89001330033010102EC30F083
:102710002FC182F40401300E8227D3EC0EF030C1B9
:1027200082F40401300E8227D3EC0EF031C182F422
:102730000401300E8227D3EC0EF032C182F4040182
:10274000300E8227D3EC0EF033C182F40401300E38
:102750008227D3EC0EF091EF29F0FC0E5CEC0BF02D
:10276000E8CF0BF003018351520AD8B4E4EF13F021
:1027700003018351720AD8B4E7EF13F003018351C8
:10278000500AD8B4EAEF13F003018351700AD8B4A9
:10279000EDEF13F003018351550AD8B4F0EF13F0B5
:1027A00003018351750AD8B4F3EF13F00301835189
:1027B000430AD8B4FCEF13F003018351630AD8B481
:1027C000FFEF13F008EF14F00B9002EF14F00B8002
:1027D00002EF14F00B9202EF14F00B8202EF14F0F0
:1027E0000B9402EF14F00B8402EF14F00B9602EF3F
:1027F00014F00B8602EF14F00B9802EF14F00B8824
:1028000002EF14F0FC0E0C6E0BC00BF045EC0BF05D
:102810000401590E826FD3EC0EF0119011921194B5
:102820001198FC0E5CEC0BF0E8CF0BF00BA01180C4
:102830000BA211820BA411840BA8118811A028EF00
:1028400014F00401520E826FD3EC0EF02DEF14F051
:102850000401720E826FD3EC0EF011A837EF14F062
:102860000401430E826FD3EC0EF03CEF14F0040130
:10287000630E826FD3EC0EF011A246EF14F0040148
:10288000500E826FD3EC0EF04BEF14F00401700E7B
:10289000826FD3EC0EF011A455EF14F00401550E25
:1028A000826FD3EC0EF05AEF14F00401750E826FB4
:1028B000D3EC0EF091EF29F004016D0E826FD3EC92
:1028C0000EF003018351300AD8B4B4EF14F00301C1
:1028D0008351310AD8B4C7EF14F003018351320A8F
:1028E000D8B4DAEF14F093EF29F004014D0E826FA3
:1028F000D3EC0EF0A0EC30F084C331F185C332F19B
:1029000086C333F10101296BADEC30F024EC30F0DB
:1029100003018351300AD8B49CEF14F003018351B2
:10292000310AD8B4A4EF14F003018351320AD8B4A9
:10293000ACEF14F093EF29F0FD0E0C6E00C10BF01C
:1029400045EC0BF0B4EF14F0FE0E0C6E00C10BF072
:1029500045EC0BF0C7EF14F0FF0E0C6E00C10BF04E
:1029600045EC0BF0DAEF14F00401300E826FD3EC7B
:102970000EF004012C0E826FD3EC0EF05FEC30F001
:10298000FD0E5CEC0BF0E8CF00F1EBEF14F004016E
:10299000310E826FD3EC0EF004012C0E826FD3EC5B
:1029A0000EF05FEC30F0FE0E5CEC0BF0E8CF00F1C7
:1029B000EBEF14F00401320E826FD3EC0EF05FECFB
:1029C00030F004012C0E826FD3EC0EF0FF0E5CECA5
:1029D0000BF0E8CF00F102EC30F031C182F40401D9
:1029E000300E8227D3EC0EF032C182F40401300E97
:1029F0008227D3EC0EF033C182F40401300E82271B
:102A0000D3EC0EF091EF29F003018351300AD8B4D2
:102A1000FFEF19F003018351310AD8B42CEF1BF0FA
:102A200003018351320AD8B49AEF1BF0030183519A
:102A3000330AD8B4AAEF1BF003018351340AD8B487
:102A400005EF1CF003018351350AD8B4EBEF1DF0FC
:102A500003018351360AD8B419EF1EF003018351E4
:102A6000370AD8B4D7EF17F003018351380AD8B426
:102A700075EF18F003018351460AD8B412EF1DF028
:102A8000030183514D0AD8B450EF16F0030183516E
:102A90006D0AD8B46AEF16F0030183515A0AD8B40C
:102AA000A6EF1AF003018351490AD8B419EF1FF0B9
:102AB00003018351500AD8B44BEF1EF00301835138
:102AC000540AD8B4C4EF1EF003018351630AD8B48A
:102AD0008AEF16F003018351430AD8B482EF17F04E
:102AE00003018351730AD8B488EF16F003018351B0
:102AF000610AD8B49DEF15F003018351650AD8B47B
:102B00004FEF1AF003018351450AD8B45DEF1AF074
:102B100003018351620AD8B46BEF1AF003018351A9
:102B2000420AD8B479EF1AF003018351760AD8B477
:102B300087EF1AF0D8A493EF29F004014C0E826FAE
:102B4000D3EC0EF00401610E826FD3EC0EF0A8EC12
:102B500031F004012C0E826FD3EC0EF05FEC30F0FC
:102B6000AFC500F1010102EC30F031C182F4040183
:102B7000300E8227D3EC0EF032C182F40401300E05
:102B80008227D3EC0EF033C182F40401300E822789
:102B9000D3EC0EF004012C0E826FD3EC0EF05FEC40
:102BA00030F0B0C500F1010102EC30F031C182F427
:102BB0000401300E8227D3EC0EF032C182F40401FE
:102BC000300E8227D3EC0EF033C182F40401300EB4
:102BD0008227D3EC0EF004012C0E826FD3EC0EF0A2
:102BE0005FEC30F0B1C500F1010102EC30F031C111
:102BF00082F40401300E8227D3EC0EF032C182F44D
:102C00000401300E8227D3EC0EF033C182F40401AC
:102C1000300E8227D3EC0EF004012C0E826FD3EC21
:102C20000EF05FEC30F0B2C500F1010102EC30F0C3
:102C300031C182F40401300E8227D3EC0EF032C190
:102C400082F40401300E8227D3EC0EF033C182F4FB
:102C50000401300E8227D3EC0EF004012C0E826F9B
:102C6000D3EC0EF05FEC30F0B6C500F1010102ECE0
:102C700030F031C182F40401300E8227D3EC0EF023
:102C800032C182F40401300E8227D3EC0EF033C13E
:102C900082F40401300E8227D3EC0EF047EF1EF0D1
:102CA000A0EC30F084C333F1ADEC30F024EC30F024
:102CB000200E0C6E00C10BF045EC0BF000C12FF59F
:102CC00005012F51000A06E005012F51010A02E01B
:102CD00042EC32F004014C0E826FD3EC0EF0040192
:102CE0004D0E826FD3EC0EF004012C0E826FD3ECEC
:102CF0000EF05FEC30F02FC500F102EC30F033C184
:102D000082F40401300E8227D3EC0EF047EF1EF060
:102D1000B1EF37F004014C0E826FD3EC0EF00401DA
:102D2000630E826FD3EC0EF000EC31F004012C0E38
:102D3000826FD3EC0EF09FEC16F047EF1EF05FECC5
:102D400030F0B5C500F10101003B0F0E001702EC99
:102D500030F033C182F40401300E8227D3EC0EF040
:102D6000B5C500F101010F0E0101001702EC30F0B2
:102D700033C182F40401300E8227D3EC0EF004013B
:102D80002D0E826FD3EC0EF0B4C500F10101003BB3
:102D90000F0E001702EC30F033C182F40401300E44
:102DA0008227D3EC0EF0B4C500F101010F0E010132
:102DB000001702EC30F033C182F40401300E822798
:102DC000D3EC0EF004012D0E826FD3EC0EF0B3C5E0
:102DD00000F10101003B0F0E001702EC30F033C18F
:102DE00082F40401300E8227D3EC0EF0B3C500F15B
:102DF00001010F0E0101001702EC30F033C182F423
:102E00000401300E8227D3EC0EF00401200E826FF5
:102E1000D3EC0EF0B2C500F10F0E0101001702EC69
:102E200030F033C182F40401300E8227D3EC0EF06F
:102E30000401200E826FD3EC0EF0B1C500F1010148
:102E40000101003B0F0E001702EC30F033C182F499
:102E50000401300E8227D3EC0EF0B1C500F1010160
:102E60000F0E0101001702EC30F033C182F40401AF
:102E7000300E8227D3EC0EF004013A0E826FD3ECB1
:102E80000EF0B0C500F10101003B0F0E001702EC7F
:102E900030F033C182F40401300E8227D3EC0EF0FF
:102EA000B0C500F101010F0E0101001702EC30F076
:102EB00033C182F40401300E8227D3EC0EF00401FA
:102EC0003A0E826FD3EC0EF0AFC500F10101003B6A
:102ED0000F0E001702EC30F033C182F40401300E03
:102EE0008227D3EC0EF0AFC500F101010F0E0017E1
:102EF00002EC30F033C182F40401300E8227D3ECAF
:102F00000EF0120084C3E8FF0F0BE83AE8CFB5F5E6
:102F100085C3E8FF0F0B0501B51387C3E8FF0F0B4F
:102F2000E83AE8CFB4F588C3E8FF0F0B0501B41306
:102F30008AC3E8FF0F0BE83AE8CFB3F58BC3E8FF8D
:102F40000F0B0501B3138DC3E8FF0F0BE8CFB2F5EC
:102F50008FC3E8FF0F0BE83AE8CFB1F590C3E8FF65
:102F60000F0B0501B11392C3E8FF0F0BE83AE8CF4E
:102F7000B0F593C3E8FF0F0B0501B01395C3E8FF4D
:102F80000F0BE83AE8CFAFF596C3E8FF0F0B05014A
:102F9000AF135BEC31F004014C0E826FD3EC0EF0FA
:102FA0000401430E826FD3EC0EF094EF16F0078409
:102FB00004014C0E826FD3EC0EF00401370E826FC9
:102FC000D3EC0EF004012C0E826FD3EC0EF0050151
:102FD0002E51130A06E005012E51170A0DE072EF7B
:102FE00018F00101000E006F000E016F100E026F4D
:102FF000000E036F05EF18F00101000E006F000EC8
:10300000016F000E026F010E036F02EC30F02AC157
:1030100082F40401300E8227D3EC0EF02BC182F42F
:103020000401300E8227D3EC0EF02CC182F404018F
:10303000300E8227D3EC0EF02DC182F40401300E45
:103040008227D3EC0EF02EC182F40401300E8227C9
:10305000D3EC0EF02FC182F40401300E8227D3ECA2
:103060000EF030C182F40401300E8227D3EC0EF052
:1030700031C182F40401300E8227D3EC0EF032C14C
:1030800082F40401300E8227D3EC0EF033C182F4B7
:103090000401300E8227D3EC0EF004012C0E826F57
:1030A000D3EC0EF00101100E006F000E016F000E48
:1030B000026F000E036F02EC30F031C182F40401A4
:1030C000300E8227D3EC0EF032C182F40401300EB0
:1030D0008227D3EC0EF033C182F40401300E822734
:1030E000D3EC0EF0079447EF1EF00501216B226B25
:1030F000236B246B04014C0E826FD3EC0EF00401A1
:10310000380E826FD3EC0EF004012C0E826FD3ECDC
:103110000EF00101100E006F000E016F000E026F25
:10312000000E036F02EC30F02AC182F40401300E6D
:103130008227D3EC0EF02BC182F40401300E8227DB
:10314000D3EC0EF02CC182F40401300E8227D3ECB4
:103150000EF02DC182F40401300E8227D3EC0EF064
:103160002EC182F40401300E8227D3EC0EF02FC161
:1031700082F40401300E8227D3EC0EF030C182F4C9
:103180000401300E8227D3EC0EF031C182F4040129
:10319000300E8227D3EC0EF032C182F40401300EDF
:1031A0008227D3EC0EF033C182F40401300E822763
:1031B000D3EC0EF004012C0E826FD3EC0EF025C57B
:1031C00000F126C501F127C502F128C503F101016F
:1031D000100E046F000E056F000E066F000E076FD5
:1031E00095EC2FF000C133F501C134F502C135F57E
:1031F00003C136F502EC30F02AC182F40401300E2E
:103200008227D3EC0EF02BC182F40401300E82270A
:10321000D3EC0EF02CC182F40401300E8227D3ECE3
:103220000EF02DC182F40401300E8227D3EC0EF093
:103230002EC182F40401300E8227D3EC0EF02FC190
:1032400082F40401300E8227D3EC0EF030C182F4F8
:103250000401300E8227D3EC0EF031C182F4040158
:10326000300E8227D3EC0EF032C182F40401300E0E
:103270008227D3EC0EF033C182F40401300E822792
:10328000D3EC0EF0DDEC0EF0050133674FEF19F0D3
:1032900034674FEF19F035674FEF19F0366702D0FA
:1032A000EEEF19F0129E129C21C500F122C501F12A
:1032B00023C502F124C503F1899A400EC76E200E82
:1032C000C66E9E96C69E0B0EC96EFF0E9EB602D0AF
:1032D000E82EFCD79E96C69E02C1C9FFFF0E9EB681
:1032E00002D0E82EFCD79E96C69E01C1C9FFFF0EF4
:1032F0009EB602D0E82EFCD79E96C69E00C1C9FF9E
:10330000FF0E9EB602D0E82EFCD79E96C69EC952EE
:10331000FF0E9EB602D0E82EFCD70501100E326FCC
:10332000040114EE00F080517F0BE1269E96C69EAC
:10333000C952FF0E9EB602D0E82EFCD7C9CFE7FFD8
:103340000401802B0501322F90EF19F0898A33C5D3
:1033500000F134C501F135C502F136C503F10101B3
:10336000010E046F000E056F000E066F000E076F52
:1033700064EC2FF000C133F501C134F502C135F51D
:1033800003C136F505013367CDEF19F03467CDEF92
:1033900019F03567CDEF19F0366702D0EEEF19F06E
:1033A00021C500F122C501F123C502F124C503F1B5
:1033B0000101100E046F000E056F000E066F000E67
:1033C000076F69EC2FF000C121F501C122F502C1A0
:1033D00023F503C124F5128E93EF29F00401450E65
:1033E000826FD3EC0EF004014F0E826FD3EC0EF01F
:1033F0000401460E826FD3EC0EF047EF1EF00784F7
:1034000072EC37F05FEC30F02DC500F102EC30F0DB
:1034100004014C0E826FD3EC0EF00401300E826F6B
:10342000D3EC0EF004012C0E826FD3EC0EF031C100
:1034300082F40401300E8227D3EC0EF032C182F404
:103440000401300E8227D3EC0EF033C182F4040164
:10345000300E8227D3EC0EF004012C0E826FD3ECD9
:103460000EF05FEC30F02EC500F102EC30F031C10F
:1034700082F40401300E8227D3EC0EF032C182F4C4
:103480000401300E8227D3EC0EF033C182F4040124
:10349000300E8227D3EC0EF0079447EF1EF00401A4
:1034A0004C0E826FD3EC0EF00401650E826FD3ECEC
:1034B0000EF01EEC33F047EF1EF004014C0E826F4D
:1034C000D3EC0EF00401450E826FD3EC0EF035EC18
:1034D00033F047EF1EF004014C0E826FD3EC0EF078
:1034E0000401620E826FD3EC0EF063EC33F047EF11
:1034F0001EF004014C0E826FD3EC0EF00401420E5C
:10350000826FD3EC0EF04CEC33F047EF1EF0040169
:103510004C0E826FD3EC0EF00401760E826FD3EC6A
:103520000EF004012C0E826FD3EC0EF010A807D021
:103530000401310E826FD3EC0EF047EF1EF0040150
:10354000300E826FD3EC0EF047EF1EF004014C0EEC
:10355000826FD3EC0EF004015A0E826FD3EC0EF0A2
:1035600004012C0E826FD3EC0EF072EC37F05FEC9E
:1035700030F005012E51130A06E005012E51170AFD
:103580000DE0D7EF1AF00101000E006F000E016F81
:10359000100E026F000E036FD7EF1AF00101000E3C
:1035A000006F000E016F000E026F010E036F01012C
:1035B000100E046F000E056F000E066F000E076FF1
:1035C00095EC2FF002EC30F02AC182F40401300EA9
:1035D0008227D3EC0EF02BC182F40401300E822737
:1035E000D3EC0EF02CC182F40401300E8227D3EC10
:1035F0000EF02DC182F40401300E8227D3EC0EF0C0
:103600002EC182F40401300E8227D3EC0EF02FC1BC
:1036100082F40401300E8227D3EC0EF030C182F424
:103620000401300E8227D3EC0EF031C182F4040184
:10363000300E8227D3EC0EF032C182F40401300E3A
:103640008227D3EC0EF033C182F40401300E8227BE
:10365000D3EC0EF047EF1EF0078404014C0E826F8E
:10366000D3EC0EF00401310E826FD3EC0EF00401A6
:103670002C0E826FD3EC0EF025C500F126C501F1AA
:1036800027C502F128C503F10101100E046F000ED9
:10369000056F000E066F000E076F95EC2FF002EC21
:1036A00030F02AC182F40401300E8227D3EC0EF0F0
:1036B0002BC182F40401300E8227D3EC0EF02CC112
:1036C00082F40401300E8227D3EC0EF02DC182F477
:1036D0000401300E8227D3EC0EF02EC182F40401D7
:1036E000300E8227D3EC0EF02FC182F40401300E8D
:1036F0008227D3EC0EF030C182F40401300E822711
:10370000D3EC0EF031C182F40401300E8227D3ECE9
:103710000EF032C182F40401300E8227D3EC0EF099
:1037200033C182F40401300E8227D3EC0EF00794EB
:1037300047EF1EF0078404014C0E826FD3EC0EF0AD
:103740000401320E826FD3EC0EF052EC35F0079488
:1037500047EF1EF0078438B0B0EF1BF0C3EF1BF04B
:10376000010E166E04014C0E826FD3EC0EF00401B4
:10377000330E826FD3EC0EF0AFEC35F0000E166E08
:10378000079437EF1BF0020E166EAFEC35F08B800E
:103790000501010E306F3C0E316F01015E6B5F6BF6
:1037A000606B616B626B636B646B656B666B676BA5
:1037B000686B696B536B546BCF6ACE6A0F9A0F9C20
:1037C0000F9E030E166E04014C0E826FD3EC0EF0AA
:1037D0000401330E826FD3EC0EF004012C0E826FC5
:1037E000D3EC0EF004012D0E826FD3EC0EF0040129
:1037F000310E826FD3EC0EF091EF29F0AFEC35F083
:10380000000E166E8B9093EF29F0078404014C0E86
:10381000826FD3EC0EF00401340E826FD3EC0EF005
:1038200004012C0E826FD3EC0EF0A0EC30F084C3B8
:103830002AF185C32BF186C32CF187C32DF188C3F0
:103840002EF189C32FF18AC330F18BC331F18CC3C0
:1038500032F18DC333F10101296BADEC30F024EC72
:1038600030F0100E046F000E056F000E066F000E94
:10387000076F75EC2FF000C121F501C122F502C1DF
:1038800023F503C124F525EC37F038C5AFF539C56C
:10389000B0F53AC5B1F53BC5B2F53CC5B3F53DC58C
:1038A000B4F53EC5B5F59FEC16F004012C0E826F01
:1038B000D3EC0EF03FC500F140C501F141C502F166
:1038C00042C503F10101000E046F000E056F010EE9
:1038D000066F000E076F95EC2FF002EC30F02967B1
:1038E00074EF1CF079EF1CF004012D0E826FD3EC05
:1038F0000EF030C182F40401300E8227D3EC0EF0BA
:1039000031C182F40401300E8227D3EC0EF00401A1
:103910002E0E826FD3EC0EF032C182F40401300E11
:103920008227D3EC0EF033C182F40401300E8227DB
:10393000D3EC0EF004012C0E826FD3EC0EF05FEC92
:1039400030F043C500F144C501F1BDEC2AF004019B
:103950002C0E826FD3EC0EF05FEC30F045C500F119
:1039600002EC30F031C182F40401300E8227D3EC36
:103970000EF032C182F40401300E8227D3EC0EF037
:1039800033C182F40401300E8227D3EC0EF004011F
:103990002C0E826FD3EC0EF037C5E8FFE8B806D0E6
:1039A0000401300E826FD3EC0EF005D00401310E0D
:1039B000826FD3EC0EF004012C0E826FD3EC0EF06C
:1039C00037C5E8FFE8BA06D00401300E826FD3ECA9
:1039D0000EF025D00401310E826FD3EC0EF00401FD
:1039E0002C0E826FD3EC0EF05FEC30F046C500F188
:1039F00002EC30F031C182F40401300E8227D3ECA6
:103A00000EF032C182F40401300E8227D3EC0EF0A6
:103A100033C182F40401300E8227D3EC0EF00794F8
:103A200047EF1EF0A0EC30F085C32AF186C32BF1DE
:103A300087C32CF188C32DF189C32EF18AC32FF1DE
:103A40008BC330F18CC331F18DC332F18EC333F1AE
:103A50000101296BADEC30F024EC30F00101010ED6
:103A6000046F000E056F000E066F000E076F64EC0A
:103A70002FF0100E046F000E056F000E066F000E83
:103A8000076F75EC2FF000C129F501C12AF502C1BD
:103A90002BF503C12CF5D9EC34F004014C0E826FE8
:103AA000D3EC0EF00401460E826FD3EC0EF004014D
:103AB0002C0E826FD3EC0EF025C500F126C501F166
:103AC00027C502F128C503F10101100E046F000E95
:103AD000056F000E066F000E076F95EC2FF002ECDD
:103AE00030F02AC182F40401300E8227D3EC0EF0AC
:103AF0002BC182F40401300E8227D3EC0EF02CC1CE
:103B000082F40401300E8227D3EC0EF02DC182F432
:103B10000401300E8227D3EC0EF02EC182F4040192
:103B2000300E8227D3EC0EF02FC182F40401300E48
:103B30008227D3EC0EF030C182F40401300E8227CC
:103B4000D3EC0EF031C182F40401300E8227D3ECA5
:103B50000EF032C182F40401300E8227D3EC0EF055
:103B600033C182F40401300E8227D3EC0EF047EF0C
:103B70001EF038B0BEEF1DF0020E166EAFEC35F041
:103B800000011650020AD8B4CBEF1DF0050E166ED8
:103B90003780B1EF37F08B8001015E6B5F6B606B3C
:103BA000616B626B636B646B656B666B676B686B99
:103BB000696B536B546BCF6ACE6A0F9A0F9C0F9E42
:103BC000030E166E93EF29F0AFEC35F0050E166E6E
:103BD0003780B1EF37F004014C0E826FD3EC0EF05A
:103BE0000401350E826FD3EC0EF004012C0E826FAF
:103BF000D3EC0EF05FEC30F00784B9C500F1079408
:103C000002EC30F031C182F40401300E8227D3EC93
:103C10000EF032C182F40401300E8227D3EC0EF094
:103C200033C182F40401300E8227D3EC0EF047EF4B
:103C30001EF072EC35F05FEC30F037C500F102ECAD
:103C400030F004014C0E826FD3EC0EF00401360EFE
:103C5000826FD3EC0EF004012C0E826FD3EC0EF0C9
:103C600031C182F40401300E8227D3EC0EF032C150
:103C700082F40401300E8227D3EC0EF033C182F4BB
:103C80000401300E8227D3EC0EF047EF1EF0DDEC7E
:103C90000EF093EF29F004014C0E826FD3EC0EF07E
:103CA0000401500E826FD3EC0EF004012C0E826FD3
:103CB000D3EC0EF085C32AF186C32BF187C32CF118
:103CC00088C32DF189C32EF18AC32FF18BC330F144
:103CD0008CC331F18DC332F18EC333F10101ADECF0
:103CE00030F024EC30F003018451530A0DE003015D
:103CF00084514D0A38E00401780E826FD3EC0EF047
:103D0000DDEC0EF093EF29F00401530E826FD3EC3B
:103D10000EF0250E0C6E00C10BF045EC0BF0260EDC
:103D20000C6E01C10BF045EC0BF0270E0C6E02C1BE
:103D30000BF045EC0BF0280E0C6E03C10BF045ECBC
:103D40000BF000C157F501C158F502C159F503C187
:103D50005AF500C15BF501C15CF502C15DF503C117
:103D60005EF528EF1FF004014D0E826FD3EC0EF0CC
:103D7000290E0C6E00C10BF045EC0BF000C15FF595
:103D800000C160F528EF1FF004014C0E826FD3ECE8
:103D90000EF00401540E826FD3EC0EF004012C0ED1
:103DA000826FD3EC0EF084C32AF185C32BF186C356
:103DB0002CF187C32DF188C32EF189C32FF18AC35B
:103DC00030F18BC331F18DC332F18EC333F1010178
:103DD000ADEC30F024EC30F00101000E046F000E69
:103DE000056F010E066F000E076F75EC2FF0210EA8
:103DF0000C6E00C10BF045EC0BF0220E0C6E01C1F5
:103E00000BF045EC0BF0230E0C6E02C10BF045ECF1
:103E10000BF0240E0C6E03C10BF045EC0BF000C14F
:103E200061F501C162F502C163F503C164F528EFD4
:103E30001FF004014C0E826FD3EC0EF00401490E0A
:103E4000826FD3EC0EF004012C0E826FD3EC0EF0D7
:103E5000250E5CEC0BF0E8CF00F1260E5CEC0BF0CD
:103E6000E8CF01F1270E5CEC0BF0E8CF02F1280E51
:103E70005CEC0BF0E8CF03F102EC30F0C5EC2DF078
:103E80000401730E826FD3EC0EF004012C0E826FCE
:103E9000D3EC0EF05FEC30F0290E5CEC0BF0E8CFC9
:103EA00000F102EC30F0C5EC2DF004016D0E826FD4
:103EB000D3EC0EF004012C0E826FD3EC0EF05BC538
:103EC00000F15CC501F15DC502F15EC503F102ECD4
:103ED00030F0C5EC2DF00401730E826FD3EC0EF0C0
:103EE00004012C0E826FD3EC0EF05FEC30F060C555
:103EF00000F102EC30F0C5EC2DF004016D0E826F84
:103F0000D3EC0EF004012C0E826FD3EC0EF061C5E1
:103F100000F162C501F163C502F164C503F1AEECC5
:103F200029F004012C0E826FD3EC0EF0DDEC0EF0C4
:103F300093EF29F083C32AF184C32BF185C32CF1BD
:103F400086C32DF187C32EF188C32FF189C330F1C9
:103F50008AC331F18BC332F18CC333F10101ADEC73
:103F600030F024EC30F0160E0C6E00C10BF045EC76
:103F70000BF0170E0C6E01C10BF045EC0BF0180E98
:103F80000C6E02C10BF045EC0BF0190E0C6E03C168
:103F90000BF045EC0BF000C18EF101C18FF102C1B5
:103FA00090F103C191F100C192F101C193F102C1FD
:103FB00094F103C195F17CEF20F083C32AF184C30F
:103FC0002BF185C32CF186C32DF187C32EF188C355
:103FD0002FF189C330F18AC331F18BC332F18CC325
:103FE00033F10101ADEC30F024EC30F000C18EF182
:103FF00001C18FF102C190F103C191F100C192F1B1
:1040000001C193F102C194F103C195F17CEF20F05D
:1040100083C32AF184C32BF185C32CF186C32DF110
:1040200087C32EF188C32FF189C330F18AC331F1E0
:104030008CC332F18DC333F10101ADEC30F024ECCF
:1040400030F00101000E046F000E056F010E066FC7
:10405000000E076F75EC2FF01A0E0C6E00C10BF0FE
:1040600045EC0BF01B0E0C6E01C10BF045EC0BF098
:104070001C0E0C6E02C10BF045EC0BF01D0E0C6E0D
:1040800003C10BF045EC0BF000C196F101C197F1B3
:1040900002C198F103C199F17CEF20F083C32AF1AA
:1040A00084C32BF185C32CF186C32DF187C32EF178
:1040B00088C32FF189C330F18AC331F18CC332F147
:1040C0008DC333F10101ADEC30F024EC30F001018F
:1040D000000E046F000E056F010E066F000E076FD5
:1040E00075EC2FF000C196F101C197F102C198F172
:1040F00003C199F17CEF20F0160E5CEC0BF0E8CFD9
:1041000000F1170E5CEC0BF0E8CF01F1180E5CEC3F
:104110000BF0E8CF02F1190E5CEC0BF0E8CF03F1E5
:1041200002EC30F0C5EC2DF00401730E826FD3EC7D
:104130000EF004012C0E826FD3EC0EF08EC100F154
:104140008FC101F190C102F191C103F102EC30F095
:10415000C5EC2DF00401730E826FD3EC0EF0040158
:104160002C0E826FD3EC0EF01A0E5CEC0BF0E8CF45
:1041700000F11B0E5CEC0BF0E8CF01F11C0E5CECC7
:104180000BF0E8CF02F11D0E5CEC0BF0E8CF03F171
:10419000AEEC29F004012C0E826FD3EC0EF096C128
:1041A00000F197C101F198C102F199C103F1AEECA0
:1041B00029F0DDEC0EF093EF29F00401690E826F17
:1041C000D3EC0EF004012C0E826FD3EC0EF0010143
:1041D000040E006F000E016F000E026F000E036FE1
:1041E00002EC30F02CC182F40401300E8227D3ECB3
:1041F0000EF02DC182F40401300E8227D3EC0EF0B4
:104200002EC182F40401300E8227D3EC0EF02FC1B0
:1042100082F40401300E8227D3EC0EF030C182F418
:104220000401300E8227D3EC0EF031C182F4040178
:10423000300E8227D3EC0EF032C182F40401300E2E
:104240008227D3EC0EF033C182F40401300E8227B2
:10425000D3EC0EF004012C0E826FD3EC0EF00101B2
:10426000060E006F000E016F000E026F000E036F4E
:1042700002EC30F02CC182F40401300E8227D3EC22
:104280000EF02DC182F40401300E8227D3EC0EF023
:104290002EC182F40401300E8227D3EC0EF02FC120
:1042A00082F40401300E8227D3EC0EF030C182F488
:1042B0000401300E8227D3EC0EF031C182F40401E8
:1042C000300E8227D3EC0EF032C182F40401300E9E
:1042D0008227D3EC0EF033C182F40401300E822722
:1042E000D3EC0EF004012C0E826FD3EC0EF0010122
:1042F000410E006F000E016F000E026F000E036F83
:1043000002EC30F02CC182F40401300E8227D3EC91
:104310000EF02DC182F40401300E8227D3EC0EF092
:104320002EC182F40401300E8227D3EC0EF02FC18F
:1043300082F40401300E8227D3EC0EF030C182F4F7
:104340000401300E8227D3EC0EF031C182F4040157
:10435000300E8227D3EC0EF032C182F40401300E0D
:104360008227D3EC0EF033C182F40401300E822791
:10437000D3EC0EF004012C0E826FD3EC0EF0200E65
:10438000F86EF76AF66A04010900F5CF82F4D3ECFF
:104390000EF00900F5CF82F4D3EC0EF00900F5CF52
:1043A00082F4D3EC0EF00900F5CF82F4D3EC0EF0DA
:1043B0000900F5CF82F4D3EC0EF00900F5CF82F4BA
:1043C000D3EC0EF00900F5CF82F4D3EC0EF0090027
:1043D000F5CF82F4D3EC0EF0DDEC0EF093EF29F084
:1043E0008351630AD8A491EF29F08451610AD8A4BB
:1043F00091EF29F085516C0AD8A491EF29F08651EC
:10440000410A3FE08651440A1BE08651420AD8B473
:1044100054EF22F08651350AD8B41DEF2BF08651A7
:10442000360AD8B472EF2BF08651370AD8B4DBEFD6
:104430002BF08651380AD8B439EF2CF091EF29F0DF
:104440000798079A04017A0E826FD3EC0EF00401EC
:10445000780E826FD3EC0EF00401640E826FD3EC01
:104460000EF00401550E826FD3EC0EF03DEF22F0FA
:1044700004014C0E826FD3EC0EF0DDEC0EF093EFE6
:1044800029F00788079A04017A0E826FD3EC0EF0A8
:104490000401410E826FD3EC0EF00401610E826FB5
:1044A000D3EC0EF031EF22F00798078A04017A0E60
:1044B000826FD3EC0EF00401420E826FD3EC0EF04B
:1044C0000401610E826FD3EC0EF031EF22F0010196
:1044D000666772EF22F0676772EF22F0686772EF2B
:1044E00022F0696716D001014F677EEF22F0506716
:1044F0007EEF22F051677EEF22F052670AD0010171
:10450000000E006F000E016F000E026F000E036FB1
:10451000120011B80AD00101620E046F010E056F7E
:10452000000E066F000E076F09D00101A70E046F81
:10453000020E056F000E066F000E076F66C100F1D8
:1045400067C101F168C102F169C103F164EC2FF0A8
:1045500003BF1BEF23F0119A119C0101000E046FA1
:10456000A80E056F550E066F020E076F66C100F1AB
:1045700067C101F168C102F169C103F166C18AF145
:1045800067C18BF168C18CF169C18DF164EC2FF0CA
:1045900003BF0BD00101000E8A6FA80E8B6F550E62
:1045A0008C6F020E8D6F118A119C0E0E5CEC0BF05D
:1045B000E8CF18F10F0E5CEC0BF0E8CF19F1100EFC
:1045C0005CEC0BF0E8CF1AF1110E5CEC0BF0E8CFCD
:1045D0001BF1ADEC2EF08AC104F18BC105F18CC149
:1045E00006F18DC107F164EC2FF0078271EC2EF01B
:1045F000ADEC2EF0079271EC2EF08AC100F18BC168
:1046000001F18CC102F18DC103F1079271EC2EF022
:10461000CC0E046FE00E056F870E066F050E076F58
:1046200064EC2FF000C118F101C119F102C11AF1B7
:1046300003C11BF140D013AA20EF23F0138E139A6D
:10464000119C119A0101800E006F1A0E016F060E67
:10465000026F000E036F4FC104F150C105F151C14B
:1046600006F152C107F164EC2FF003AF05D05FEC07
:1046700030F0118C119A12000E0E5CEC0BF0E8CFAA
:1046800018F10F0E5CEC0BF0E8CF19F1100E5CEC9A
:104690000BF0E8CF1AF1110E5CEC0BF0E8CF1BF138
:1046A0004FC100F150C101F151C102F152C103F1FA
:1046B000078271EC2EF018C100F119C101F11AC185
:1046C00002F11BC103F112000784BAC166F1BBC13C
:1046D00067F1BCC168F1BDC169F14BC14FF14CC17B
:1046E00050F14DC151F14EC152F157C159F158C16C
:1046F0005AF107940101666785EF23F0676785EF3C
:1047000023F0686785EF23F0696716D001014F67D2
:1047100091EF23F0506791EF23F0516791EF23F071
:1047200052670AD00101000E006F000E016F000EEB
:10473000026F000E036F120011B80AD00101620E61
:10474000046F010E056F000E066F000E076F09D093
:104750000101A70E046F020E056F000E066F000E1A
:10476000076F66C100F167C101F168C102F169C15B
:1047700003F164EC2FF003BF1DEF24F00101000EE4
:10478000046FA80E056F550E066F020E076F66C107
:1047900000F167C101F168C102F169C103F166C1AD
:1047A0008AF167C18BF168C18CF169C18DF164EC4C
:1047B0002FF003BF09D00101000E8A6FA80E8B6F86
:1047C000550E8C6F020E8D6FADEC2EF000C104F112
:1047D00001C105F102C106F103C107F1000E006F2E
:1047E000A00E016F980E026F7B0E036F95EC2FF0F9
:1047F00000C118F101C119F102C11AF103C11BF185
:10480000000E006FA00E016F980E026F7B0E036FFB
:104810008AC104F18BC105F18CC106F18DC107F18C
:1048200095EC2FF018C104F119C105F11AC106F178
:104830001BC107F164EC2FF012000101A80E006FFC
:10484000610E016F000E026F000E036F4FC104F185
:1048500050C105F151C106F152C107F164EC2FF0CE
:1048600003AF0AD00101A80E006F610E016F000EA8
:10487000026F000E036F00D0C80E006FAF0E016F05
:10488000000E026F000E036F4FC104F150C105F11D
:1048900051C106F152C107F175EC2FF0120004016D
:1048A000730E826FD3EC0EF004012C0E826FD3ECEA
:1048B0000EF0078462C166F163C167F164C168F1FB
:1048C00065C169F14BC14FF14CC150F14DC151F17E
:1048D0004EC152F157C159F158C15AF1079475ECC4
:1048E00024F0DDEC0EF093EF29F066C100F167C112
:1048F00001F168C102F169C103F1010102EC30F07C
:10490000C5EC2DF00401630E826FD3EC0EF00401B0
:104910002C0E826FD3EC0EF04FC100F150C101F1AB
:1049200051C102F152C103F1010102EC30F0C5ECBA
:104930002DF00401660E826FD3EC0EF004012C0EF4
:10494000826FD3EC0EF05FEC30F059C100F15AC128
:1049500001F1010102EC30F0C5EC2DF00401740E00
:10496000826FD3EC0EF0120010820401530E826F9E
:10497000D3EC0EF004012C0E826FD3EC0EF083C347
:104980002AF184C32BF185C32CF186C32DF187C393
:104990002EF188C32FF189C330F18AC331F18BC363
:1049A00032F18CC333F10101ADEC30F024EC30F086
:1049B00000C166F101C167F102C168F103C169F18B
:1049C0008EC32AF18FC32BF190C32CF191C32DF12B
:1049D00092C32EF193C32FF194C330F195C331F1FB
:1049E00096C332F197C333F10101ADEC30F024EC02
:1049F00030F000C14FF101C150F102C151F103C1CA
:104A000052F1A0EC30F099C32FF19AC330F19BC35F
:104A100031F19CC332F19DC333F10101ADEC30F0B3
:104A200024EC30F000C159F101C15AF175EC24F0C9
:104A300004012C0E826FD3EC0EF02FEF25F0118EB7
:104A40001CA002D01CAE108C1BBE02D01BA4108E6A
:104A500003018251520A02E10F8201D00F9282516A
:104A6000750A02E1108401D010948251550A02E1C6
:104A7000108601D010968351310A03E1138213840A
:104A800002D01392139403018351660A01E056D0B9
:104A90000401660E826FD3EC0EF004012C0E826FBF
:104AA000D3EC0EF064EC23F002EC30F02AC182F477
:104AB0000401300E8227D3EC0EF02BC182F40401E6
:104AC000300E8227D3EC0EF02CC182F40401300E9C
:104AD0008227D3EC0EF02DC182F40401300E822720
:104AE000D3EC0EF02EC182F40401300E8227D3ECF9
:104AF0000EF02FC182F40401300E8227D3EC0EF0A9
:104B000030C182F40401300E8227D3EC0EF031C1A3
:104B100082F40401300E8227D3EC0EF032C182F40D
:104B20000401300E8227D3EC0EF033C182F404016D
:104B3000300E8227D3EC0EF091EF29F011A003D0B4
:104B400011A401D01084078410B208EF26F010A43D
:104B5000ECEF25F0BAC166F1BBC167F1BCC168F1E9
:104B6000BDC169F1BEC16AF1BFC16BF1C0C16CF1D9
:104B7000C1C16DF1C2C16EF1C3C16FF1C4C170F1A9
:104B8000C5C171F1C6C172F1C7C173F1C8C174F179
:104B9000C9C175F1CAC176F1CBC177F1CCC178F149
:104BA000CDC179F1CEC17AF1CFC17BF1D0C17CF119
:104BB000D1C17DF1D2C17EF1D3C17FF1D4C180F1E9
:104BC000D5C181F1D6C182F1D7C183F1D8C184F1B9
:104BD000D9C185F1F4EF25F062C166F163C167F1D7
:104BE00064C168F165C169F1BAC186F1BBC187F1E1
:104BF000BCC188F1BDC189F14BC14FF14CC150F12D
:104C00004DC151F14EC152F157C159F158C15AF13C
:104C100007940FA02AEF26F00101966717EF26F000
:104C2000976717EF26F0986717EF26F099671BEF45
:104C300026F02AEF26F067EC22F096C104F197C126
:104C400005F198C106F199C107F164EC2FF003BF9B
:104C500057EF29F067EC22F00101000E046F000EFF
:104C6000056F010E066F000E076F95EC2FF011A077
:104C70002AD011A228D002EC30F0296701D005D04B
:104C800004012D0E826FD3EC0EF030C182F40401CA
:104C9000300E8227D3EC0EF031C182F40401300EC5
:104CA0008227D3EC0EF032C182F40401300E822749
:104CB000D3EC0EF033C182F40401300E8227D3EC22
:104CC0000EF0DDEC0EF012A8C5D012981DC01EF03B
:104CD0001E3A1E42070E1E1600011E50000AD8B4CE
:104CE000F6EF26F000011E50010AD8B482EF26F03C
:104CF00000011E50020AD8B480EF26F028EF27F0FA
:104D000028EF27F05FEC30F02DC001F12EC000F14C
:104D1000D89001330033D890013300330101630E82
:104D2000046F000E056F000E066F000E076F95EC06
:104D30002FF0280E046F000E056F000E066F000E98
:104D4000076F64EC2FF000C130F05FEC30F02BC047
:104D500001F1019F019D2CC000F10101A40E046F1F
:104D6000000E056F000E066F000E076F95EC2FF01A
:104D700000C12FF000C104F101C105F102C106F12B
:104D800003C107F1640E006F000E016F000E026F89
:104D9000000E036F64EC2FF0050E046F000E056F1C
:104DA000000E066F000E076F95EC2FF000C104F1A6
:104DB00001C105F102C106F103C107F15FEC30F05A
:104DC00030C000F164EC2FF000C131F031C0E8FFD9
:104DD000050F305C03E78A8428EF27F031C0E8FF35
:104DE0000A0F305C01E68A9428EF27F000C124F115
:104DF00001C125F102C126F103C127F15FEC30F0BA
:104E000065EC30F01D501F0BE8CF00F10101640E7E
:104E1000046F000E056F000E066F000E076F75EC35
:104E20002FF024C104F125C105F126C106F127C1E7
:104E300007F164EC2FF003BF02D08A9401D08A847A
:104E400024C100F125C101F126C102F127C103F1FE
:104E500093EF29F000C124F101C125F102C126F12F
:104E600003C127F110AE4DD0109E00C108F101C161
:104E700009F102C10AF103C10BF102EC30F030C1BB
:104E8000E2F131C1E3F132C1E4F133C1E5F108C12E
:104E900000F109C101F10AC102F10BC103F10101E5
:104EA0006C0E046F070E056F000E066F000E076F85
:104EB00064EC2FF003BF04D00101550EE66F1CD047
:104EC00008C100F109C101F10AC102F10BC103F1EE
:104ED0000101A40E046F060E056F000E066F000E92
:104EE000076F64EC2FF003BF04D001017F0EE66F63
:104EF00003D00101FF0EE66F1F8E11AE57EF29F0B0
:104F0000119E24C100F125C101F126C102F127C182
:104F100003F111A005D011A203D00FB057EF29F073
:104F200010A49AEF27F00401750E826FD3EC0EF0F7
:104F30009FEF27F00401720E826FD3EC0EF0040194
:104F40002C0E826FD3EC0EF002EC30F02967AEEF3E
:104F500027F00401200E826FB1EF27F004012D0E1F
:104F6000826FD3EC0EF030C182F40401300E822740
:104F7000D3EC0EF031C182F40401300E8227D3EC61
:104F80000EF004012E0E826FD3EC0EF032C182F4CB
:104F90000401300E8227D3EC0EF033C182F40401F9
:104FA000300E8227D3EC0EF004016D0E826FD3EC2D
:104FB0000EF004012C0E826FD3EC0EF04FC100F105
:104FC00050C101F151C102F152C103F1010102ECE2
:104FD00030F0C5EC2DF00401480E826FD3EC0EF0DA
:104FE00004017A0E826FD3EC0EF004012C0E826F56
:104FF000D3EC0EF066C100F167C101F168C102F1A6
:1050000069C103F1010102EC30F0C5EC2DF004019F
:10501000630E826FD3EC0EF004012C0E826FD3EC82
:105020000EF066C100F167C101F168C102F169C10A
:1050300003F101010A0E046F000E056F000E066FEA
:10504000000E076F75EC2FF0000E046F120E056F47
:10505000000E066F000E076F95EC2FF002EC30F09B
:105060002AC182F40401300E8227D3EC0EF02BC14A
:1050700082F40401300E8227D3EC0EF02CC182F4AE
:105080000401300E8227D3EC0EF02DC182F404010E
:10509000300E8227D3EC0EF02EC182F40401300EC4
:1050A0008227D3EC0EF02FC182F40401300E822748
:1050B000D3EC0EF030C182F40401300E8227D3EC21
:1050C0000EF004012E0E826FD3EC0EF031C182F48B
:1050D0000401300E8227D3EC0EF032C182F40401B9
:1050E000300E8227D3EC0EF033C182F40401300E6F
:1050F0008227D3EC0EF00401730E826FD3EC0EF016
:1051000004012C0E826FD3EC0EF05FEC30F059C12D
:1051100000F15AC101F1BDEC2AF013A2DFEF28F033
:1051200004012C0E826FD3EC0EF086C166F187C1AC
:1051300067F188C168F189C169F167EC22F001016A
:10514000000E046F000E056F010E066F000E076F54
:1051500095EC2FF002EC30F02967B4EF28F0040151
:10516000200E826FB7EF28F004012D0E826FD3EC72
:105170000EF030C182F40401300E8227D3EC0EF021
:1051800031C182F40401300E8227D3EC0EF0040109
:105190002E0E826FD3EC0EF032C182F40401300E79
:1051A0008227D3EC0EF033C182F40401300E822743
:1051B000D3EC0EF004016D0E826FD3EC0EF013A44D
:1051C00006EF29F004012C0E826FD3EC0EF013AC25
:1051D000F4EF28F00401500E826FD3EC0EF0139C14
:1051E0001398139A06EF29F013AE01EF29F004018A
:1051F000460E826FD3EC0EF0139E1398139A06EFAF
:1052000029F00401530E826FD3EC0EF038B01DEF7D
:1052100029F004012C0E826FD3EC0EF08BB018EF46
:1052200029F00401440E826FD3EC0EF01DEF29F03B
:105230000401530E826FD3EC0EF00FB223EF29F06E
:105240000FA055EF29F004012C0E826FD3EC0EF065
:10525000200EF86EF76AF66A04010900F5CF82F4B1
:10526000D3EC0EF00900F5CF82F4D3EC0EF0090078
:10527000F5CF82F4D3EC0EF00900F5CF82F4D3EC35
:105280000EF00900F5CF82F4D3EC0EF00900F5CF53
:1052900082F4D3EC0EF00900F5CF82F4D3EC0EF0DB
:1052A0000900F5CF82F4D3EC0EF0DDEC0EF00F9098
:1052B000109E129893EF29F00401630E826FD3ECD5
:1052C0000EF004012C0E826FD3EC0EF099EC29F055
:1052D00004012C0E826FD3EC0EF00CEC2AF00401CA
:1052E0002C0E826FD3EC0EF088EC2AF004012C0E09
:1052F000826FD3EC0EF00101F80E006FCD0E016F3E
:10530000660E026F030E036FAEEC29F004012C0E43
:10531000826FD3EC0EF09EEC2AF0DDEC0EF093EFF2
:1053200029F0DDEC0EF00301C26B07901092A2EFA2
:105330002CF0D8900E0E5CEC0BF0E8CF00F10F0EC5
:105340005CEC0BF0E8CF01F1100E5CEC0BF0E8CF59
:1053500002F1110E5CEC0BF0E8CF03F10101000E3D
:10536000046F000E056F010E066F000E076F95ECBF
:105370002FF002EC30F02AC182F40401300E8227B3
:10538000D3EC0EF02BC182F40401300E8227D3EC53
:105390000EF02CC182F40401300E8227D3EC0EF003
:1053A0002DC182F40401300E8227D3EC0EF02EC101
:1053B00082F40401300E8227D3EC0EF02FC182F468
:1053C0000401300E8227D3EC0EF030C182F40401C8
:1053D000300E8227D3EC0EF031C182F40401300E7E
:1053E0008227D3EC0EF004012E0E826FD3EC0EF068
:1053F00032C182F40401300E8227D3EC0EF033C1A7
:1054000082F40401300E8227D3EC0EF004016D0EFD
:10541000826FD3EC0EF01200120E5CEC0BF0E8CFB2
:1054200000F1130E5CEC0BF0E8CF01F1140E5CEC14
:105430000BF0E8CF02F1150E5CEC0BF0E8CF03F1B6
:1054400001010A0E046F000E056F000E066F000EBC
:10545000076F75EC2FF0000E046F120E056F000E33
:10546000066F000E076F95EC2FF002EC30F02AC1AA
:1054700082F40401300E8227D3EC0EF02BC182F4AB
:105480000401300E8227D3EC0EF02CC182F404010B
:10549000300E8227D3EC0EF02DC182F40401300EC1
:1054A0008227D3EC0EF02EC182F40401300E822745
:1054B000D3EC0EF02FC182F40401300E8227D3EC1E
:1054C0000EF030C182F40401300E8227D3EC0EF0CE
:1054D00004012E0E826FD3EC0EF031C182F4040170
:1054E000300E8227D3EC0EF032C182F40401300E6C
:1054F0008227D3EC0EF033C182F40401300E8227F0
:10550000D3EC0EF00401730E826FD3EC0EF0120098
:105510000A0E5CEC0BF0E8CF00F10B0E5CEC0BF02C
:10552000E8CF01F10C0E5CEC0BF0E8CF02F10D0EB0
:105530005CEC0BF0E8CF03F1BDEF2AF0060E5CEC5B
:105540000BF0E8CF00F1070E5CEC0BF0E8CF01F1B7
:10555000080E5CEC0BF0E8CF02F1090E5CEC0BF0EE
:10556000E8CF03F1BDEF2AF001015FEC30F00784D2
:1055700057C100F158C101F107940101E80E046F11
:10558000800E056F000E066F000E076F75EC2FF092
:10559000000E046F040E056F000E066F000E076FFD
:1055A00095EC2FF0880E046F130E056F000E066F3A
:1055B000000E076F64EC2FF00A0E046F000E056FEB
:1055C000000E066F000E076F95EC2FF002EC30F026
:1055D00001012967F1EF2AF00401200E826FF4EF38
:1055E0002AF004012D0E826FD3EC0EF030C182F44C
:1055F0000401300E8227D3EC0EF031C182F4040195
:10560000300E8227D3EC0EF032C182F40401300E4A
:105610008227D3EC0EF004012E0E826FD3EC0EF035
:1056200033C182F40401300E8227D3EC0EF0040162
:10563000430E826FD3EC0EF0120087C32AF188C3A9
:105640002BF189C32CF18AC32DF18BC32EF18CC3AE
:105650002FF18DC330F18EC331F190C332F191C37C
:1056600033F10101296BADEC30F024EC30F0010195
:10567000000E046F000E056F010E066F000E076F1F
:1056800075EC2FF00E0E0C6E00C10BF045EC0BF01C
:105690000F0E0C6E01C10BF045EC0BF0100E0C6EF2
:1056A00002C10BF045EC0BF0110E0C6E03C10BF0B8
:1056B00045EC0BF004017A0E826FD3EC0EF004017E
:1056C0002C0E826FD3EC0EF00401350E826FD3ECFA
:1056D0000EF004012C0E826FD3EC0EF099EC29F041
:1056E0003DEF22F087C32AF188C32BF189C32CF147
:1056F0008AC32DF18BC32EF18CC32FF18DC330F1F2
:105700008EC331F190C332F191C333F10101296BA2
:10571000ADEC30F024EC30F0880E046F130E056F02
:10572000000E066F000E076F69EC2FF0000E046F7D
:10573000040E056F000E066F000E076F75EC2FF05C
:105740000101E80E046F800E056F000E066F000E5B
:10575000076F95EC2FF00A0E0C6E00C10BF045ECB4
:105760000BF00B0E0C6E01C10BF045EC0BF00C0EA8
:105770000C6E02C10BF045EC0BF00D0E0C6E03C16C
:105780000BF045EC0BF004017A0E826FD3EC0EF0B7
:1057900004012C0E826FD3EC0EF00401360E826FE2
:1057A000D3EC0EF004012C0E826FD3EC0EF088ECDB
:1057B0002AF03DEF22F087C32AF188C32BF189C379
:1057C0002CF18AC32DF18BC32EF18CC32FF18DC325
:1057D00030F18FC331F190C332F191C333F1010144
:1057E000ADEC30F024EC30F0000E046F120E056FBB
:1057F000000E066F000E076F75EC2FF001010A0E08
:10580000046F000E056F000E066F000E076F95EC1B
:105810002FF0120E0C6E00C10BF045EC0BF0130EC6
:105820000C6E01C10BF045EC0BF0140E0C6E02C1B6
:105830000BF045EC0BF0150E0C6E03C10BF045ECB4
:105840000BF004017A0E826FD3EC0EF004012C0EE3
:10585000826FD3EC0EF00401370E826FD3EC0EF0A2
:1058600004012C0E826FD3EC0EF00CEC2AF03DEF0D
:1058700022F087C32AF188C32BF189C32CF18AC394
:105880002DF18BC32EF18CC32FF18DC330F18EC35C
:1058900031F190C332F191C333F10101296BADECC9
:1058A00030F024EC30F0880E046F130E056F000EFC
:1058B000066F000E076F69EC2FF0000E046F040EE8
:1058C000056F000E066F000E076F75EC2FF00101DB
:1058D000E80E046F800E056F000E066F000E076F56
:1058E00095EC2FF0060E0C6E00C10BF045EC0BF0A2
:1058F000070E0C6E01C10BF045EC0BF0080E0C6EA0
:1059000002C10BF045EC0BF0090E0C6E03C10BF05D
:1059100045EC0BF004017A0E826FD3EC0EF004011B
:105920002C0E826FD3EC0EF00401380E826FD3EC94
:105930000EF004012C0E826FD3EC0EF09EEC2AF0D8
:105940003DEF22F007A815EF2DF00101800E006F4A
:105950001A0E016F060E026F000E036F4BC104F1A9
:105960004CC105F14DC106F14EC107F164EC2FF0B9
:1059700003BF5BEF2DF0BFEC2DF04BC100F14CC12C
:1059800001F14DC102F14EC103F1078271EC2EF01D
:1059900018C104F119C105F11AC106F11BC107F1C3
:1059A000F80E006FCD0E016F660E026F030E036FCF
:1059B00064EC2FF00E0E0C6E00C10BF045EC0BF0FA
:1059C0000F0E0C6E01C10BF045EC0BF0100E0C6EBF
:1059D00002C10BF045EC0BF0110E0C6E03C10BF085
:1059E00045EC0BF0078401015FEC30F057C100F18A
:1059F00058C101F107940A0E0C6E00C10BF045EC82
:105A00000BF00B0E0C6E01C10BF045EC0BF00C0E05
:105A10000C6E02C10BF045EC0BF00D0E0C6E03C1C9
:105A20000BF045EC0BF05BEF2DF007AA5BEF2DF0D0
:105A3000078401015FEC30F057C100F158C101F15A
:105A40000794060E0C6E00C10BF045EC0BF0070E30
:105A50000C6E01C10BF045EC0BF0080E0C6E02C190
:105A60000BF045EC0BF0090E0C6E03C10BF045EC8E
:105A70000BF0078462C100F163C101F164C102F15E
:105A800065C103F10794120E0C6E00C10BF045ECDA
:105A90000BF0130E0C6E01C10BF045EC0BF0140E65
:105AA0000C6E02C10BF045EC0BF0150E0C6E03C131
:105AB0000BF045EC0BF00798079A0401805181190F
:105AC0007F0B0DE09EA8FED714EE00F081517F0BF6
:105AD000E126E750812B0F01AD6E5DEF2DF0050142
:105AE0002F51010A0FE081AA87EF2DF005012F51F8
:105AF000000AD8B4B1EF37F000011650050AD8B447
:105B0000B1EF37F081B887EF2DF0A8EC31F001EF5D
:105B10000EF018C100F119C101F11AC102F11BC147
:105B200003F1000E046F000E056F010E066F000EEC
:105B3000076F95EC2FF029A1B4EF2DF02051D8B4C8
:105B4000B4EF2DF018C100F119C101F11AC102F131
:105B50001BC103F1000E046F000E056F0A0E066FE5
:105B6000000E076F95EC2FF0120001010451001395
:105B700005510113065102130751031312000101CD
:105B8000186B196B1A6B1B6B12002AC182F404018B
:105B9000300E8227D3EC0EF02BC182F40401300EBC
:105BA0008227D3EC0EF02CC182F40401300E822740
:105BB000D3EC0EF02DC182F40401300E8227D3EC19
:105BC0000EF02EC182F40401300E8227D3EC0EF0C9
:105BD0002FC182F40401300E8227D3EC0EF030C1C5
:105BE00082F40401300E8227D3EC0EF031C182F42E
:105BF0000401300E8227D3EC0EF032C182F404018E
:105C0000300E8227D3EC0EF033C182F40401300E43
:105C10008227D3EC0EF012002FC182F40401300E63
:105C20008227D3EC0EF030C182F40401300E8227BB
:105C3000D3EC0EF031C182F40401300E8227D3EC94
:105C40000EF032C182F40401300E8227D3EC0EF044
:105C500033C182F40401300E8227D3EC0EF012001F
:105C6000060E216E060E226E060E236E212E36EFD4
:105C70002EF0222E36EF2EF0232E36EF2EF08B84D0
:105C8000020E216E020E226E020E236E212E46EFB0
:105C90002EF0222E46EF2EF0232E46EF2EF08B9480
:105CA0001200FF0E226E22C023F0030E216E8B84A1
:105CB000212E57EF2EF0030E216E232E57EF2EF0DC
:105CC0008B9422C023F0030E216E212E65EF2EF05F
:105CD000030E216E233E65EF2EF0222E53EF2EF0A1
:105CE00012000101005305E1015303E1025301E1F8
:105CF000002B34EC2FF05FEC30F03951006F3A514B
:105D0000016F420E046F4B0E056F000E066F000E02
:105D1000076F75EC2FF000C104F101C105F102C15C
:105D200006F103C107F118C100F119C101F11AC14F
:105D300002F11BC103F107B2A2EF2EF069EC2FF0C4
:105D4000A4EF2EF064EC2FF000C118F101C119F19D
:105D500002C11AF103C11BF112005FEC30F059C10E
:105D600000F15AC101F1060E5CEC0BF0E8CF04F132
:105D7000070E5CEC0BF0E8CF05F1080E5CEC0BF0C5
:105D8000E8CF06F1090E5CEC0BF0E8CF07F164EC0C
:105D90002FF000C124F101C125F102C126F103C198
:105DA00027F1290E046F000E056F000E066F000E1E
:105DB000076F75EC2FF0EE0E046F430E056F000EAB
:105DC000066F000E076F69EC2FF024C104F125C1A6
:105DD00005F126C106F127C107F175EC2FF000C1CE
:105DE0001CF101C11DF102C11EF103C11FF1120E10
:105DF0005CEC0BF0E8CF04F1130E5CEC0BF0E8CF99
:105E000005F1140E5CEC0BF0E8CF06F1150E5CEC1E
:105E10000BF0E8CF07F10D0E006F000E016F000EC2
:105E2000026F000E036F75EC2FF0180E046F000E5A
:105E3000056F000E066F000E076F95EC2FF01CC16A
:105E400004F11DC105F11EC106F11FC107F169EC86
:105E50002FF06A0E046F2A0E056F000E066F000EFB
:105E6000076F64EC2FF01200BF0EFA6E200E3A6F2F
:105E7000396BD8900037013702370337D8B045EF78
:105E80002FF03A2F3AEF2FF039073A070353D8B4DF
:105E900012000331070B80093F6F03390F0B010F0D
:105EA000396F80EC5FF0406F390580EC5FF0405D4A
:105EB000405F396B3F33D8B0392739333FA95AEFA8
:105EC0002FF0405139271200010184EC30F0D8B096
:105ED0001200010103510719346F47EC30F0D890DC
:105EE0000751031934AF800F12000101346B6BECC2
:105EF00030F0D8A081EC30F0D8B0120056EC30F081
:105F00005FEC30F01F0E366F97EC30F00B35D8B0E9
:105F100047EC30F0D8A00335D8B01200362F84EF0C
:105F20002FF034B16EEC30F012000101346B0451EB
:105F30000511061107110008D8A06BEC30F0D8A0AD
:105F400081EC30F0D8B01200086B096B0A6B0B6B58
:105F500097EC30F01F0E366F97EC30F007510B5D69
:105F6000D8A4BFEF2FF006510A5DD8A4BFEF2FF0E1
:105F70000551095DD8A4BFEF2FF00451085DD8A0EA
:105F8000D2EF2FF00451085F0551D8A0053D095FFD
:105F90000651D8A0063D0A5F0751D8A0073D0B5F08
:105FA000D8900081362FACEF2FF034B16EEC30F08A
:105FB000346B6BEC30F0D8909BEC30F007510B5DFC
:105FC000D8A4EFEF2FF006510A5DD8A4EFEF2FF021
:105FD0000551095DD8A4EFEF2FF00451085DD8A05A
:105FE000FEEF2FF0003FFEEF2FF0013FFEEF2FF00E
:105FF000023FFEEF2FF0032BD8B4120034B16EEC49
:1060000030F012000101346B6BEC30F0D8B01200AC
:10601000A0EC30F0200E366F00370137023703371F
:1060200011EE33F00A0E376FE7360A0EE75CD8B090
:10603000E76EE552372F14EF30F0362F0CEF30F0CB
:1060400034B12981D890120001010A0E346F200E5C
:10605000366F11EE29F03451376F0A0ED890E652A0
:10606000D8B0E726E732372F2FEF30F00333023373
:1060700001330033362F29EF30F0E750FF0FD8A05F
:106080000335D8B0120029B16EEC30F01200045183
:1060900000270551D8B0053D01270651D8B0063D6F
:1060A00002270751D8B0073D032712000051086F9F
:1060B0000151096F02510A6F03510B6F1200010168
:1060C000006B016B026B036B12000101046B056B2B
:1060D000066B076B12000335D8A012000351800B2A
:1060E000001F011F021F031F003F7EEF30F0013F22
:1060F0007EEF30F0023F7EEF30F0032B342B032590
:1061000012000735D8A012000751800B041F051F8D
:10611000061F071F043F94EF30F0053F94EF30F067
:10612000063F94EF30F0072B342B07251200003781
:10613000013702370337083709370A370B371200A0
:106140000101296B2A6B2B6B2C6B2D6B2E6B2F6B2C
:10615000306B316B326B336B120001012A510F0B24
:106160002A6F2B510F0B2B6F2C510F0B2C6F2D51B6
:106170000F0B2D6F2E510F0B2E6F2F510F0B2F6FFB
:1061800030510F0B306F31510F0B316F32510F0BFC
:10619000326F33510F0B336F120000C124F101C174
:1061A00025F102C126F103C127F104C100F105C1A7
:1061B00001F106C102F107C103F124C104F125C1B7
:1061C00005F126C106F127C107F1120010A806D07B
:1061D0008994000EC76E220EC66E05D08984000E0B
:1061E000C76E220EC66E050EE82EFED7120010A84E
:1061F00002D0898401D08994050EE82EFED71200C2
:10620000E6EC30F09E96C69E000EC96EFF0E9EB65E
:1062100002D0E82EFCD79E96C69E000EC96EFF0ED9
:106220009EB602D0E82EFCD7C9CFAFF59E96C69E8B
:10623000000EC96EFF0E9EB602D0E82EFCD7C9CF65
:10624000B0F59E96C69E000EC96EFF0E9EB602D099
:10625000E82EFCD7C9CFB1F59E96C69E000EC96E3A
:10626000FF0E9EB602D0E82EFCD7C9CFB2F59E969F
:10627000C69E000EC96EFF0E9EB602D0E82EFCD759
:10628000C9CFB3F59E96C69E000EC96EFF0E9EB690
:1062900002D0E82EFCD7C9CFB4F59E96C69E000E5C
:1062A000C96EFF0E9EB602D0E82EFCD7C9CFB5F559
:1062B000F7EC30F01200E6EC30F09E96C69E800EB1
:1062C000C96EFF0E9EB602D0E82EFCD79E96C69EE3
:1062D000AFC5C9FFFF0E9EB602D0E82EFCD79E9632
:1062E000C69EB0C5C9FFFF0E9EB602D0E82EFCD7F1
:1062F0009E96C69EB1C5C9FFFF0E9EB602D0E82E7F
:10630000FCD79E96C69EB2C5C9FFFF0E9EB602D0B0
:10631000E82EFCD79E96C69EB3C5C9FFFF0E9EB65B
:1063200002D0E82EFCD79E96C69EB4C5C9FFFF0ECC
:106330009EB602D0E82EFCD79E96C69EB5C5C9FF74
:10634000FF0E9EB602D0E82EFCD7F7EC30F012001C
:10635000E6EC30F09E96C69E070EC96EFF0E9EB606
:1063600002D0E82EFCD79E96C69E000EC96EFF0E88
:106370009EB602D0E82EFCD7C9CFAFF59E96C69E3A
:10638000000EC96EFF0E9EB602D0E82EFCD7C9CF14
:10639000B0F59E96C69E000EC96EFF0E9EB602D048
:1063A000E82EFCD7C9CFB1F59E96C69E000EC96EE9
:1063B000FF0E9EB602D0E82EFCD7C9CFB2F5F7EC9F
:1063C00030F0E6EC30F09E96C69E25C0C9FFFF0E69
:1063D0009EB602D0E82EFCD79E96C69E000EC96ED1
:1063E000FF0E9EB602D0E82EFCD7C9CFB6F5F7EC6B
:1063F00030F01200E6EC30F09E96C69E870EC96E15
:10640000FF0E9EB602D0E82EFCD79E96C69EAFC564
:10641000C9FFFF0E9EB602D0E82EFCD79E96C69E00
:10642000B0C5C9FFFF0E9EB602D0E82EFCD79E96DF
:10643000C69EB1C5C9FFFF0E9EB602D0E82EFCD79E
:106440009E96C69EB2C5C9FFFF0E9EB602D0E82E2C
:10645000FCD7F7EC30F0E6EC30F09E96C69E26C0F6
:10646000C9FFFF0E9EB602D0E82EFCD79E96C69EB0
:10647000B6C5C9FFFF0E9EB602D0E82EFCD7F7ECDA
:1064800030F01200E6EC30F09E96C69E870EC96E84
:10649000FF0E9EB602D0E82EFCD79E96C69E000E3A
:1064A000C96EFF0E9EB602D0E82EFCD79E96C69E01
:1064B000800EC96EFF0E9EB602D0E82EFCD79E96C7
:1064C000C69E800EC96EFF0E9EB602D0E82EFCD787
:1064D0009E96C69E800EC96EFF0E9EB602D0E82E16
:1064E000FCD7F7EC30F01200E6EC30F09E96C69E3A
:1064F000870EC96EFF0E9EB602D0E82EFCD79E9680
:10650000C69E000EC96EFF0E9EB602D0E82EFCD7C6
:106510009E96C69E000EC96EFF0E9EB602D0E82E55
:10652000FCD79E96C69E800EC96EFF0E9EB602D008
:10653000E82EFCD79E96C69E800EC96EFF0E9EB6B4
:1065400002D0E82EFCD7F7EC30F0120010A817D0DC
:10655000E6EC30F09E96C69E8F0EC96EFF0E9EB67C
:1065600002D0E82EFCD79E96C69E000EC96EFF0E86
:106570009EB602D0E82EFCD7F7EC30F01200A8EC63
:1065800031F0120010A82DD0E6EC30F09E96C69E99
:1065900026C0C9FFFF0E9EB602D0E82EFCD79E96FD
:1065A000C69E450EC96EFF0E9EB602D0E82EFCD7E1
:1065B000F7EC30F0E6EC30F09E96C69E8F0EC96E7A
:1065C000FF0E9EB602D0E82EFCD79E96C69E000E09
:1065D000C96EFF0E9EB602D0E82EFCD7F7EC30F065
:1065E0001200E6EC30F09E96C69E26C0C9FFFF0E54
:1065F0009EB602D0E82EFCD79E96C69E010EC96EAE
:10660000FF0E9EB602D0E82EFCD7F7EC30F0E6EC99
:1066100030F09E96C69E910EC96EFF0E9EB602D0B9
:10662000E82EFCD79E96C69EA50EC96EFF0E9EB69E
:1066300002D0E82EFCD7F7EC30F01200E6EC30F098
:106640009E96C69E26C0C9FFFF0E9EB602D0E82EBB
:10665000FCD79E96C69E810EC96EFF0E9EB602D0D6
:10666000E82EFCD7F7EC30F01200E6EC30F09E9606
:10667000C69E26C0C9FFFF0E9EB602D0E82EFCD7EC
:106680009E96C69E010EC96EFF0E9EB602D0E82EE3
:10669000FCD7F7EC30F01200E6EC30F09E96C69E88
:1066A000910EC96EFF0E9EB602D0E82EFCD79E96C4
:1066B000C69EA50EC96EFF0E9EB602D0E82EFCD770
:1066C000F7EC30F01200E6EC30F09E96C69E910E8C
:1066D000C96EFF0E9EB602D0E82EFCD79E96C69ECF
:1066E000000EC96EFF0E9EB602D0E82EFCD7F7EC66
:1066F00030F012000501256B266B276B286B899AF9
:10670000400EC76E200EC66E9E96C69E030EC96EC4
:10671000FF0E9EB602D0E82EFCD79E96C69E27C5D9
:10672000C9FFFF0E9EB602D0E82EFCD79E96C69EED
:1067300026C5C9FFFF0E9EB602D0E82EFCD79E9656
:10674000C69E25C5C9FFFF0E9EB602D0E82EFCD717
:106750009E96C69EC952FF0E9EB602D0E82EFCD76A
:10676000898A0F01C950FF0A01E1120005012E516B
:10677000130A05E005012E51170A0CE0120005016D
:10678000F00E256FFF0E266F0F0E276F000E286F7D
:10679000D3EF33F00501F00E256FFF0E266FFF0ECD
:1067A000276F000E286F899A400EC76E200EC66EA6
:1067B0009E96C69E030EC96EFF0E9EB602D0E82EB0
:1067C000FCD79E96C69E27C5C9FFFF0E9EB602D077
:1067D000E82EFCD79E96C69E26C5C9FFFF0E9EB624
:1067E00002D0E82EFCD79E96C69E25C5C9FFFF0E97
:1067F0009EB602D0E82EFCD79E96C69EC952FF0ECA
:106800009EB602D0E82EFCD7898A0F01C950FF0A34
:106810001DE005012E51130A05E005012E51170A4E
:106820000BE012000501000E256F000E266F100E02
:10683000276F000E286F12000501000E256F000E55
:10684000266F000E276F010E286F12000501256BC1
:10685000266B276B286B05012E51130A05E00501F5
:106860002E51170A0CE012000501000E216F000ED8
:10687000226F080E236F000E246F48EF34F00501DD
:10688000000E216F000E226F800E236F000E246F0A
:1068900021C500F122C501F123C502F124C503F190
:1068A00025C504F126C505F127C506F128C507F160
:1068B000B5EC2DF000C125F501C126F502C127F583
:1068C00003C128F5899A400EC76E200EC66E9E96AB
:1068D000C69E030EC96EFF0E9EB602D0E82EFCD7F0
:1068E0009E96C69E27C5C9FFFF0E9EB602D0E82E13
:1068F000FCD79E96C69E26C5C9FFFF0E9EB602D047
:10690000E82EFCD79E96C69E25C5C9FFFF0E9EB6F3
:1069100002D0E82EFCD79E96C69EC952FF0E9EB6A8
:1069200002D0E82EFCD7898AC950FF0A08E104C1C9
:1069300025F505C126F506C127F507C128F5D8902C
:10694000050124332333223321332151F00B216FEE
:1069500005012167B3EF34F02267B3EF34F023670A
:10696000B3EF34F0246748EF34F00501100E25270B
:10697000E86A2623E86A2723E86A28231200E86ADF
:1069800005012E51130A06E005012E51170A0BE0EE
:10699000020E120005012851000A03E12751F00BF5
:1069A00007E0010E120005012851000A01E0010E66
:1069B000120029C500F12AC501F12BC502F12CC531
:1069C00003F125C504F126C505F127C506F128C543
:1069D00007F164EC2FF003BF1200BFEC34F0D8A431
:1069E00051EF35F0899A400EC76E200EC66E9E9606
:1069F000C69E060EC96EFF0E9EB602D0E82EFCD7CC
:106A0000898A899A9E96C69E020EC96EFF0E9EB610
:106A100002D0E82EFCD79E96C69E27C5C9FFFF0E62
:106A20009EB602D0E82EFCD79E96C69E26C5C9FF0C
:106A3000FF0E9EB602D0E82EFCD79E96C69E25C5B8
:106A4000C9FFFF0E9EB602D0E82EFCD79E96C69ECA
:106A5000000EC96EFF0E9EB602D0E82EFCD7898AC2
:106A6000899A9E96C69E050EC96EFF0E9EB602D0EE
:106A7000E82EFCD79E96C69EC952FF0E9EB602D047
:106A8000E82EFCD7C9B03AEF35F0898A0501100E1F
:106A90002527E86A2623E86A2723E86A2823D9EF0E
:106AA00034F01200899A400EC76E200EC66E9E9674
:106AB000C69E060EC96EFF0E9EB602D0E82EFCD70B
:106AC000898A899A9E96C69EC70EC96EFF0E9EB68B
:106AD00002D0E82EFCD7898A0501256B266B276B2F
:106AE000286B1200899A400EC76E200EC66E9E96C5
:106AF000C69E050EC96EFF0E9EB602D0E82EFCD7CC
:106B00009E96C69EC952FF0E9EB602D0E82EFCD7B6
:106B1000C9CF37F5898A1200899A400EC76E200EB8
:106B2000C66E9E96C69EB90EC96EFF0E9EB602D068
:106B3000E82EFCD7898A1200899A400EC76E200E73
:106B4000C66E9E96C69EAB0EC96EFF0E9EB602D056
:106B5000E82EFCD7898AFF0EE82EFED71200BFEC84
:106B600034F0D8A41200899A400EC76E200EC66E6B
:106B70009E96C69E030EC96EFF0E9EB602D0E82EEC
:106B8000FCD79E96C69E27C5C9FFFF0E9EB602D0B3
:106B9000E82EFCD79E96C69E26C5C9FFFF0E9EB660
:106BA00002D0E82EFCD79E96C69E25C5C9FFFF0ED3
:106BB0009EB602D0E82EFCD79E96C69EC952FF0E06
:106BC0009EB602D0E82EFCD7898A0F01C950FF0A71
:106BD000D8A423EF37F00501FE0E376F37A03799A1
:106BE00000EC31F0AFC538F5B0C539F5B1C53AF5AF
:106BF000B2C53BF5B3C53CF5B4C53DF5B5C53EF5ED
:106C00000784BAC166F1BBC167F1BCC168F1BDC1FF
:106C100069F14BC14FF14CC150F14DC151F14EC121
:106C200052F157C159F158C15AF100011650010AE9
:106C3000D8B429EF36F000011650020AD8B442EF5A
:106C400036F000011650040AD8B458EF36F023EF9E
:106C500037F00501000E466F8BA0379B67EC22F0E2
:106C600000C1DAF101C1DBF102C1DCF103C1DDF1E8
:106C700000C13FF501C140F502C141F503C142F534
:106C800091EF36F067EC22F000C1DAF101C1DBF1DF
:106C900002C1DCF103C1DDF164EC23F000C1DEF1DF
:106CA00001C1DFF102C1E0F103C1E1F123EF37F0EF
:106CB000379BDAC13FF5DBC140F5DCC141F5DDC1F1
:106CC00042F564EC23F0DEC104F1DFC105F1E0C15F
:106CD00006F1E1C107F164EC2FF003AF75EF36F078
:106CE0000501000E466F91EF36F0720E046F030E31
:106CF000056F000E066F000E076F95EC2FF003670F
:106D00008AEF36F002678AEF36F001678AEF36F0D5
:106D10008FEF36F00501FF0E466F91EF36F000C1A0
:106D200046F5050161679CEF36F062679CEF36F02F
:106D300063679CEF36F06467A0EF36F0B5EF36F08E
:106D4000DAC100F1DBC101F1DCC102F1DDC103F107
:106D500061C504F162C505F163C506F164C507F1BB
:106D600064EC2FF003BF23EF37F059C143F55AC14C
:106D700044F5B9C545F50501110E326F899A400EEB
:106D8000C76E200EC66E9E96C69E060EC96EFF0E7C
:106D90009EB602D0E82EFCD7898A899A9E96C69E16
:106DA000020EC96EFF0E9EB602D0E82EFCD79E964C
:106DB000C69E27C5C9FFFF0E9EB602D0E82EFCD79F
:106DC0009E96C69E26C5C9FFFF0E9EB602D0E82E2F
:106DD000FCD79E96C69E25C5C9FFFF0E9EB602D063
:106DE000E82EFCD725EE37F0322F02D003EF37F034
:106DF0009E96C69EDECFC9FFFF0E9EB602D0E82E3D
:106E0000FCD7F4EF36F0898A899A9E96C69E050EC5
:106E1000C96EFF0E9EB602D0E82EFCD79E96C69E87
:106E2000C952FF0E9EB602D0E82EFCD7C9B00EEFB5
:106E300037F0898A0501100E2527E86A2623E86ABB
:106E40002723E86A28230794120021C500F122C5F0
:106E500001F123C502F124C503F1899A400EC76EE2
:106E6000200EC66E9E96C69E0B0EC96EFF0E9EB677
:106E700002D0E82EFCD79E96C69E02C1C9FFFF0E27
:106E80009EB602D0E82EFCD79E96C69E01C1C9FFD1
:106E9000FF0E9EB602D0E82EFCD79E96C69E00C17D
:106EA000C9FFFF0E9EB602D0E82EFCD79E96C69E66
:106EB000C952FF0E9EB602D0E82EFCD725EE37F061
:106EC0000501100E326F9E96C69EC952FF0E9EB6E9
:106ED00002D0E82EFCD7C9CFDEFF322F63EF37F0A8
:106EE000898A1200899A400EC76E200EC66E9E9641
:106EF000C69E900EC96EFF0E9EB602D0E82EFCD73D
:106F00009E96C69E000EC96EFF0E9EB602D0E82E5B
:106F1000FCD79E96C69E000EC96EFF0E9EB602D08E
:106F2000E82EFCD79E96C69E000EC96EFF0E9EB63A
:106F300002D0E82EFCD79E96C69EC952FF0E9EB682
:106F400002D0E82EFCD7C9CF2DF59E96C69EC95219
:106F5000FF0E9EB602D0E82EFCD7C9CF2EF5898A47
:106F600012008B9030EC2EF0B9C5E8FFD70802E391
:106F700030EC2EF0B9C5E8FFC80802E330EC2EF083
:106F8000B9C5E8FFB90802E330EC2EF0B9C5E8FF57
:106F9000AA0802E330EC2EF0B9C5E8FF9B0802E333
:106FA00030EC2EF08CEC35F0F29CF29E8B94C69A6D
:106FB000C2909482948C720ED36ED3A4FED789961D
:106FC0008A909390F29AF2949D909E909D929E92B8
:106FD000F298F292A6EC32F0FF0EE8CF00F0E82E25
:106FE000FED7002EFCD7F290F286815081A8FBEFED
:106FF00037F0F29E0300700ED36EF296F290010EFF
:0C700000376E038051EC2EF091EF0BF086
:10BF0000E844F926000C160C2B0C3F0C520C640C68
:10BF1000760C860C960CA50CB30CC10CCF0CDC0C6B
:06BF2000E80CF40C000C1B
:0200000400F00A
:0100C800FE39
:00000001FF
